:100000000C946B430C94B64A0C9488430C9488432C
:100010000C9488430C9488430C948A430C94884332
:100020000C9488430C9488430C9488430C94884324
:100030000C9488430C9488430C9488430C94884314
:100040000C949E4A0C9488430C9488430C948843E7
:100050000C9488430C9488430C9488430C948843F4
:100060000C9488430C9488430C9488430C948843E4
:100070000C9488430C9488430C94884318F09FE5B3
:1000800018F09FE518F09FE518F09FE518F09FE540
:100090000000A0E114F09FE514F09FE52801F0BFF7
:1000A0004002F0BF4402F0BF4802F0BF4C02F0BF74
:1000B0005002F0BF5402F0BF0000000008009FE5AE
:1000C00008209FE5002082E01EFF2FE1F87DF0BFB1
:1000D0007864010024009FE50010A0E3001080E593
:1000E000C01080E518109FE5081080E5FF10A0E320
:1000F000C41080E50010A0E3101080E51EFF2FE182
:10010000000300F8FFFF0100000000EA1B0E00EAF8
:1001100028008FE2000C90E800A08AE001704AE21B
:1001200000B08BE00B005AE1140E000A0F00BAE891
:1001300014E04FE2010013E303F0471013FF2FE137
:100140003C0100004C0100000000A0E30050A0E1D1
:10015000B4009FE5000055E3CF10E003FF10E0136B
:10016000001080E50010E0E3041080E50E12E0E3EB
:10017000081080E594109F0594109F150C1080E5E1
:1001800090009FE50110A0E3081080E588F09FE54E
:1001900074009FE5000055E3CE10E003FE10E0136D
:1001A000001080E574109FE5FE1F91E870509FE5F8
:1001B000D1F021E300D045E2D2F021E301DC45E2B9
:1001C000D7F021E302DC45E2DBF021E302DC45E28B
:1001D000D3F021E302DC45E2130000EB3C0000EB2E
:1001E00010F021E30EDD45E20108A0E334109FE5A5
:1001F000242091E50F28C2E3002082E1242081E53C
:100200000220A0E32C2081E5BEFFFFEA000000F8F9
:10021000F01FF42FF31FF42F000C00F81401F0BFAF
:100220002801F0BFF8FFF1BF000100F81C009FE5B6
:1002300018109FE518209FE5021041E014209FE56B
:10024000010050E101208114FCFFFF1A1EFF2FE185
:10025000F8FFF1BF881D0000D0D0ADDE0000000027
:10026000000000000000000000000000000000008E
:10027000000000000000000000000000E479F0BF72
:10028000F8FFF1BF04000000102100C000000000D2
:10029000000000000000000000000000000000005E
:1002A000000000000000000000000000000000004E
:1002B0000000000000000000000000007C1104EAC3
:1002C000AF4F04EA791104EA771104EA884F04EA8F
:1002D000781104EA7EFFFFEAD24F04EA9A1104EA99
:1002E0007847C046991104EA7847C046711400EA7D
:1002F000711400EA6F1400EA6FFFFFEAB83304EAF2
:100300009A1104EA911104EA7847C046901400EA71
:100310007847C046951104EA4B1400EACE1400EA6F
:10032000E61400EA041500EA953304EA933204EA7D
:10033000D32904EAC54F04EA9D3004EA091E04EA01
:10034000973304EAEC1504EAA41304EA2E1504EA30
:100350002B1404EAB41404EACC1504EA991704EA4D
:10036000E31704EAFC1000EAC51304EACF2D04EAFF
:100370003D1704EA430E00EA0E0E00EA8C1404EA6C
:100380004D3E04EA151704EAF41504EA972C04EA32
:10039000E33804EA841304EA661304EAA61304EAC1
:1003A000232D04EABB1404EA021204EA9F0D00EABA
:1003B000981104EAF52B04EABA2B04EAF23F04EAA6
:1003C0003E1504EA5E2E04EAED2C04EAA72C04EAAA
:1003D000F73104EA033204EA7D1104EA852E04EAC7
:1003E000553004EAC53E04EA0C0E00EAD42B04EAB8
:1003F000651704EAD13804EA313904EAEA2C04EA40
:10040000C92B04EACE3B04EAC60D00EA7E3B04EAAF
:10041000D31104EA1E1804EA151504EA131804EAB5
:10042000CB1204EA081804EA3A1404EA993804EAF8
:10043000AF3B04EA633904EA523904EAB61304EA2A
:10044000400E00EABA1604EA0F1304EA451404EA5F
:10045000661104EAF11204EA8C1204EADC3004EAC0
:10046000D23504EA543104EA7847C04600C09FE51B
:100470001CFF2FE1A36D00C07847C04600C09FE578
:100480001CFF2FE1C16900C07847C04600C09FE54E
:100490001CFF2FE1716B00C07847C04600C09FE58C
:1004A0001CFF2FE1F53EF0BF7847C04600C09FE536
:1004B0001CFF2FE1FB6D00C07847C04600C09FE5E0
:1004C0001CFF2FE1656A00C07847C04600C09FE569
:1004D0001CFF2FE1316600C07847C04600C09FE591
:1004E0001CFF2FE1916600C07847C04600C09FE521
:1004F0001CFF2FE14D6A00C07847C04600C09FE551
:100500001CFF2FE14942F0BF7847C04600C09FE57D
:100510001CFF2FE1C96900C07847C04600C09FE5B5
:100520001CFF2FE1917500C07847C04600C09FE5D1
:100530001CFF2FE1357600C07847C04600C09FE51C
:100540001CFF2FE1A17400C07847C04600C09FE5A2
:100550001CFF2FE1ED6900C07847C04600C09FE551
:100560001CFF2FE1C17000C07847C04600C09FE566
:100570001CFF2FE11D6A00C07847C04600C09FE500
:100580001CFF2FE1F97000C07847C04600C09FE50E
:100590001CFF2FE1316D00C07847C04600C09FE5C9
:1005A0001CFF2FE1217400C07847C04600C09FE5C2
:1005B0001CFF2FE1F942F0BF7847C04600C09FE51D
:1005C0001CFF2FE1B57200C07847C04600C09FE510
:1005D0001CFF2FE1697600C07847C04600C09FE548
:1005E0001CFF2FE1436D00C07847C04600C09FE567
:1005F0001CFF2FE1476D00C07847C04600C09FE553
:100600001CFF2FE1257000C07847C04600C09FE561
:100610001CFF2FE14D6D00C07847C04600C09FE52C
:100620001CFF2FE18D7200C07847C04600C09FE5D7
:100630001CFF2FE16D7300C07847C04600C09FE5E6
:100640001CFF2FE1297200C07847C04600C09FE51B
:100650001CFF2FE1C97100C07847C04600C09FE56C
:100660001CFF2FE1357300C07847C04600C09FE5EE
:100670001CFF2FE1BD7200C07847C04600C09FE557
:100680001CFF2FE1FD7200C07847C04600C09FE507
:100690001CFF2FE1ED6A00C07847C0463D1300EA19
:1006A0007847C04600C09FE51CFF2FE1F56400C0FD
:1006B0007847C04600C09FE51CFF2FE1657000C071
:1006C0007847C04600C09FE51CFF2FE1216E00C0A7
:1006D0007847C04600C09FE51CFF2FE1516E00C067
:1006E0007847C04600C09FE51CFF2FE1517500C050
:1006F0007847C04600C09FE51CFF2FE1F56B00C0A6
:100700007847C04600C09FE51CFF2FE14D6C00C03C
:100710007847C0461F1300EA7847C04600C09FE5EF
:100720001CFF2FE1517200C07847C04600C09FE512
:100730001CFF2FE1F17100C07847C04600C09FE563
:100740001CFF2FE1D97300C07847C04600C09FE569
:100750001CFF2FE1B542F0BF7847C04600C09FE5BF
:100760001CFF2FE1353EF0BF7847C04600C09FE533
:100770001CFF2FE1A13DF0BF7847C04600C09FE5B8
:100780001CFF2FE1C96B00C07847C04600C09FE541
:100790001CFF2FE1C140F0BF7847C04600C09FE575
:1007A0001CFF2FE1C57600C07847C04600C09FE51A
:1007B0001CFF2FE1517600C07847C046CC3A04EACE
:1007C0007847C0463C3D04EA7847C04600C09FE5F4
:1007D0001CFF2FE13D7600C07847C0468A3A04EA04
:1007E0007847C04600C09FE51CFF2FE1197100C08B
:1007F0007847C04600C09FE51CFF2FE15541F0BF80
:100800007847C04600C09FE51CFF2FE1ED6E00C099
:100810007847C04600C09FE51CFF2FE1916F00C0E4
:100820007847C04600C09FE51CFF2FE1596500C016
:100830007847C046CB1C04EA7847C046613804EAD2
:1008400000C09FE51CFF2FE18F7D00C000C09FE529
:100850001CFF2FE1117F00C000C09FE51CFF2FE1AE
:10086000537F00C0280F00EAC04604EA1F1704EABD
:100870004F2A04EA802A04EA702A04EA412A04EA98
:10088000C54504EA7847C04600C09FE51CFF2FE13C
:100890003B7D00C07847C04600C09FE51CFF2FE1AC
:1008A000BB7C00C07847C046743E04EA7847C04627
:1008B000324104EA7847C046B23D04EA7847C04670
:1008C00000C09FE51CFF2FE19F7F00C07847C04616
:1008D0003C4104EA7847C0467C4204EA7847C04677
:1008E000944104EA7847C046C94104EA7847C046C3
:1008F000CE4104EA7847C046E74104EA7847C0465B
:10090000FF4104EA7847C0468D3A04EA7847C0467A
:100910004D3004EA7847C04600C09FE51CFF2FE138
:10092000BD7E00C07847C04600C09FE51CFF2FE198
:10093000398700C07847C04600C09FE51CFF2FE103
:100940008B7D00C07847C04600C09FE51CFF2FE1AB
:10095000B58800C07847C04600C09FE51CFF2FE166
:100960002D8000C07847C04600C09FE51CFF2FE1E6
:100970008F7D00C07847C04600C09FE51CFF2FE177
:10098000737D00C07847C04600C09FE51CFF2FE183
:10099000358100C07847C04600C09FE51CFF2FE1AD
:1009A000D58200C07847C04600C09FE51CFF2FE1FC
:1009B0002D7D00C07847C04600C09FE51CFF2FE199
:1009C0009D7C00C07847C04600C09FE51CFF2FE11A
:1009D000FD7C00C07847C04600C09FE51CFF2FE1AA
:1009E000D37C00C07847C04600C09FE51CFF2FE1C4
:1009F000E57C00C07847C04600C09FE51CFF2FE1A2
:100A0000C37C00C07847C04600C09FE51CFF2FE1B3
:100A1000437D00C07847C04600C09FE51CFF2FE122
:100A2000698800C07847C04600C09FE51CFF2FE1E1
:100A3000B37F00C07847C04600C09FE51CFF2FE190
:100A4000418800C07847C04600C09FE51CFF2FE1E9
:100A5000CB7C00C07847C04600C09FE51CFF2FE15B
:100A6000537F00C07847C04600C09FE51CFF2FE1C0
:100A7000317D00C07847C04600C09FE51CFF2FE1D4
:100A8000B97D00C07847C04600C09FE51CFF2FE13C
:100A90008D8800C07847C04600C09FE51CFF2FE14D
:100AA0003B8700C07847C04600C09FE51CFF2FE190
:100AB000CD7E00C07847C04600C09FE51CFF2FE1F7
:100AC000E97E00C07847C04600C09FE51CFF2FE1CB
:100AD000977E00C07847C04600C09FE51CFF2FE10D
:100AE000E98800C07847C04600C09FE51CFF2FE1A1
:100AF0003D8900C07847C04600C09FE51CFF2FE13C
:100B0000117F00C07847C04600C09FE51CFF2FE161
:100B10009B7F00C07847C04600C09FE51CFF2FE1C7
:100B2000AB7F00C07847C04600C09FE51CFF2FE1A7
:100B3000AF7F00C07847C04600C09FE51CFF2FE193
:100B4000897C00C07847C046EC3C04EA7847C04640
:100B500000C09FE51CFF2FE1038700C07847C04617
:100B600000C09FE51CFF2FE1F18600C07847C0461A
:100B700000C09FE51CFF2FE1D17E00C07847C04632
:100B800000C09FE51CFF2FE11D8900C07847C046CB
:100B9000553004EA7847C046343004EA7847C04606
:100BA00000C09FE51CFF2FE1418700C07847C04689
:100BB00000C09FE51CFF2FE13F8700C07847C0467B
:100BC00000C09FE51CFF2FE1458700C07847C04665
:100BD00000C09FE51CFF2FE1F97F00C07847C046A9
:100BE000683704EA0A2204EA162004EA822104EAA9
:100BF000924504EA132204EA944504EAE51100EA66
:100C0000152E04EACD2004EAC82004EAC32004EA31
:100C1000B72004EA412E04EAAD2004EA002204EAE7
:100C20006E2104EA7F2E04EA772E04EA113E04EADC
:100C3000002004EA332204EAA92004EA642104EA39
:100C4000CE2504EA242504EA742404EABF2004EA39
:100C50008A0E00EAAD2204EAE02204EA413104EA05
:100C6000791B04EA470F04EA473104EABE2604EA86
:100C7000FC2204EAF62204EAD32204EA630E00EA24
:100C8000E62204EAD43704EA6F2F04EA872804EA4C
:100C9000D42604EA2E2704EADA2604EACC2704EA5A
:100CA000020F00EA1E0F00EAC10E00EA920E00EAEF
:100CB000572804EAB92704EAC82604EA432704EAC5
:100CC0005B2804EAE02704EA282804EA7847C046BB
:100CD000072804EA7847C0461D2704EA7847C0463B
:100CE000082704EA7847C046102804EA7847C04637
:100CF0008A2704EA7847C046CD2704EA7847C046E9
:100D0000262804EA7847C046E42704EA7847C04624
:100D1000DE2704EA7847C0465F2704EA7847C046E2
:100D2000FD2604EA9F2304EAC12304EAF82304EA27
:100D3000242404EAB62904EA352604EADD2B04EA71
:100D4000A82B04EA8D2B04EA1D2B04EAEE2A04EA00
:100D5000492B04EA032B04EA302B04EA102C04EAA2
:100D60008B2C04EA942C04EA3B2C04EAB02C04EA11
:100D7000A42D04EA822C04EA3D0E00EAD72C04EAF2
:100D80007D2C04EA802C04EA821100EA3E0E00EA7F
:100D9000E22F04EA1F3004EA5B2F04EA132F04EA6F
:100DA000EA3604EA293604EA213604EA753004EA10
:100DB000543004EA703904EA550F00EA543604EA64
:100DC000DF3004EAF12E04EA202E04EACB1504EA0F
:100DD000A40D00EA090C00EA402F04EA262F04EAD9
:100DE0005A3604EA1C3704EA5C2204EAE02D04EADD
:100DF0008C2D04EAE60E00EA711B04EA1D3104EAB8
:100E0000933104EA873104EA313204EAAC3104EA6E
:100E10007847C0464A3204EA7847C0469D3104EA22
:100E20007847C0461E0E00EA7847C0467A3704EA83
:100E30007847C046263104EA323904EA8F3204EAA0
:100E40006F3204EA473304EAA63204EA193304EAAB
:100E50005B2C04EA353404EAD90404EADE0404EA2B
:100E6000C73504EA9D3404EA683504EA6C3404EAC0
:100E7000893504EAFF3304EA943304EA4F3304EA81
:100E8000103404EACB3304EA673304EA023404EA98
:100E9000BA3304EA623304EACA3504EA073504EADD
:100EA0002D3404EACA3404EAF83304EA973304EA36
:100EB000493304EA803304EA7B3604EAD32C04EA9B
:100EC000991A04EAA91A04EA452C04EA632C04EAF4
:100ED0003D3604EAA02E04EA9A2C04EAD72B04EA51
:100EE000FF2C04EA262D04EA033604EA152D04EA51
:100EF000942E04EAFC2C04EAFB3504EAC53504EA26
:100F00002F3D04EA603804EA813804EAB83704EA7D
:100F1000383904EAB03B04EA0A3B04EA7B3904EAC4
:100F2000D74404EA860F00EA6C4C04EA403704EA2E
:100F3000673704EA113804EA233804EA0B3904EA73
:100F4000DF4404EAF84404EA8A4C04EA5E4C04EA0A
:100F5000793704EA844C04EA763804EA833A04EAEE
:100F6000353A04EA373B04EA923904EA393D04EAA7
:100F70002F3904EA443D04EAB13904EA4B3A04EA61
:100F80006F3904EA243904EA5B3B04EAB33804EA23
:100F9000393904EAFD3804EA453804EA263804EA17
:100FA000E23B04EAD63C04EA3E4C04EA173C04EA7D
:100FB000DD3E04EA254204EAC73D04EA8C1E04EA49
:100FC0009B2504EABE3E04EA493F04EAF23D04EAF6
:100FD000B03E04EAF33E04EA9C3E04EA223F04EAFF
:100FE000713E04EA034104EA7A4104EAF14104EA69
:100FF000BE4104EA3D3D04EA4E3D04EAAE2504EA62
:10100000283E04EA934104EA394104EA863D04EAB1
:10101000BF1E04EA7847C04600C09FE51CFF2FE1D1
:10102000151D01C07847C04600C09FE51CFF2FE199
:101030004B1E01C07847C04600C09FE51CFF2FE152
:101040001D1C01C07847C04600C09FE51CFF2FE172
:10105000451C01C07847C04600C09FE51CFF2FE13A
:10106000E11801C07847C04600C09FE51CFF2FE192
:101070007D1E01C07847C04600C09FE51CFF2FE1E0
:10108000D51E01C07847C04600C09FE51CFF2FE178
:10109000011C01C07847C04600C09FE51CFF2FE13E
:1010A000791C01C07847C04600C09FE51CFF2FE1B6
:1010B000E11C01C07847C04600C09FE51CFF2FE13E
:1010C000A51B01C07847C04600C09FE51CFF2FE16B
:1010D000351901C07847C046343204EA7847C04623
:1010E000410E00EA7847C0465E0E00EA7847C046E7
:1010F000603204EA7847C04600C09FE51CFF2FE13C
:10110000ED1801C07847C04600C09FE51CFF2FE1E5
:10111000D11B01C07847C046A52E04EA7847C046D7
:10112000B02E04EA7847C046D23C04EA8F4304EA72
:101130007847C046620E00EA7847C04600C09FE587
:101140001CFF2FE1E51801C07847C046421100EAB4
:101150007847C04600C09FE51CFF2FE1511901C030
:101160007847C04600C09FE51CFF2FE1891A01C0E7
:101170007847C04600C09FE51CFF2FE11D1E01C03F
:101180007847C04600C09FE51CFF2FE1551F01C0F6
:101190007847C046911507EA7847C046701507EAB8
:1011A0007847C046151507EA7847C04600C09FE556
:1011B0001CFF2FE1691F01C07847C046381507EAB8
:1011C0007847C046A41507EA7847C04600C09FE5A7
:1011D0001CFF2FE14943F0BF7847C04600C09FE5A0
:1011E0001CFF2FE10D7800C0B72E04EA290D00EA9C
:1011F000A52E04EA2D4404EA7847C04600C09FE5C6
:101200001CFF2FE10D3E01C07847C04600C09FE59E
:101210001CFF2FE1613F01C07847C04600C09FE539
:101220001CFF2FE1A93A01C07847C04600C09FE5E6
:101230001CFF2FE1E551F0BF7847C04600C09FE595
:101240001CFF2FE1F13401C07847C04600C09FE584
:101250001CFF2FE17B3701C07847C04600C09FE5E7
:101260001CFF2FE1553801C07847C04600C09FE5FC
:101270001CFF2FE1653701C07847C04600C09FE5DD
:101280001CFF2FE1F14CF0BF7847C04600C09FE53E
:101290001CFF2FE1F12C01C07847C04600C09FE53C
:1012A0001CFF2FE1092801C07847C04600C09FE518
:1012B0001CFF2FE1FF3701C07847C04600C09FE503
:1012C0001CFF2FE1054EF0BF7847C04600C09FE5E8
:1012D0001CFF2FE1CD3701C07847C04600C09FE515
:1012E0001CFF2FE1B92901C07847C04600C09FE527
:1012F0001CFF2FE1C13801C07847C04600C09FE500
:101300001CFF2FE10F3901C07847C04600C09FE5A0
:101310001CFF2FE1DD3801C07847C04600C09FE5C3
:101320001CFF2FE1313401C07847C04600C09FE563
:101330001CFF2FE1FD2F01C07847C04600C09FE58C
:101340001CFF2FE1A12F01C07847C04600C09FE5D8
:101350001CFF2FE19D2601C07847C04600C09FE5D5
:101360001CFF2FE12B3901C07847C0469F1000EACF
:101370007847C04600C09FE51CFF2FE10D52F0BF2B
:101380007847C04600C09FE51CFF2FE12D2C01C00F
:101390007847C04600C09FE51CFF2FE1113A01C00D
:1013A0007847C04600C09FE51CFF2FE1052B01C018
:1013B0007847C046C71904EA7847C046D31904EAFB
:1013C0007847C046B41904EA7847C04600C09FE594
:1013D0001CFF2FE1253A01C07847C04600C09FE5B9
:1013E0001CFF2FE11F3A01C07847C04600C09FE5AF
:1013F0001CFF2FE15D3901C07847C04600C09FE562
:101400001CFF2FE15D2B01C07847C04600C09FE55F
:101410001CFF2FE1853801C07847C04600C09FE51A
:101420001CFF2FE1973701C07847C04600C09FE5F9
:101430001CFF2FE1C12C01C07847C04600C09FE5CA
:101440001CFF2FE1493A01C07847C04600C09FE524
:101450001CFF2FE1E53301C07847C046FD7604EA62
:101460007847C04600C09FE51CFF2FE16B3E01C0DE
:101470007847C04600C09FE51CFF2FE14D3E01C0EC
:101480007847C046807704EA7847C0460D7704EA7B
:101490007847C04600C09FE51CFF2FE1313801C0EE
:1014A0007847C046947804EA7847C04600C09FE574
:1014B0001CFF2FE1ED3201C07847C04600C09FE518
:1014C0001CFF2FE1512D01C07847C04600C09FE5A9
:1014D0001CFF2FE1A54FF0BF7847C04600C09FE535
:1014E0001CFF2FE1C150F0BF7847C04600C09FE508
:1014F0001CFF2FE1B52801C07847C04600C09FE51A
:101500001CFF2FE1E12401C07847C04600C09FE5E1
:101510001CFF2FE1F53C01C07847C0462F7904EA53
:101520007847C046CE7804EA7847C04600C09FE5B9
:101530001CFF2FE1C53E01C07847C04600C09FE5B3
:101540001CFF2FE1833E01C07847C04600C09FE5E5
:101550001CFF2FE1D93D01C07847C04600C09FE580
:101560001CFF2FE1693A01C07847C04600C09FE5E3
:101570001CFF2FE1353C01C07847C04600C09FE505
:101580001CFF2FE1112301C07847C04600C09FE532
:101590001CFF2FE18D52F0BF7847C04600C09FE589
:1015A0001CFF2FE1E93E01C0020900EA2E4304EAD4
:1015B0001D4B04EABB3A04EAEF2604EAEF2604EAEC
:1015C000B54A04EAB54A04EA971D04EA971D04EAFD
:1015D000002F04EA002F04EA7847C04600C09FE5C8
:1015E0001CFF2FE13D2101C07847C04600C09FE5A8
:1015F0001CFF2FE1572001C07847C04600C09FE57F
:101600001CFF2FE10B2101C07847C04600C09FE5B9
:101610001CFF2FE1492001C07847C04600C09FE56C
:101620001CFF2FE1F11F01C07847C04600C09FE5B5
:101630001CFF2FE1072101C07847C04600C09FE58D
:101640001CFF2FE1E72001C07847C04600C09FE59E
:101650001CFF2FE1D92001C07847C04600C09FE59C
:101660001CFF2FE16D2001C07847C04600C09FE5F8
:101670001CFF2FE1352601C07847C04600C09FE51A
:101680001CFF2FE1892501C07847C04600C09FE5B7
:101690001CFF2FE1B18400C07847C04600C09FE521
:1016A0001CFF2FE1418500C07847C04600C09FE580
:1016B0001CFF2FE1B18000C07847C04600C09FE505
:1016C0001CFF2FE1118100C07847C04600C09FE594
:1016D0001CFF2FE1358600C07847C04600C09FE55B
:1016E0001CFF2FE15D8300C07847C04600C09FE526
:1016F0001CFF2FE1658000C07847C04600C09FE511
:101700001CFF2FE1E58500C07847C04600C09FE57B
:101710001CFF2FE1618400C07847C04600C09FE5F0
:101720001CFF2FE1E98500C07847C04600C09FE557
:101730001CFF2FE1458000C07847C04600C09FE5F0
:101740001CFF2FE1558000C07847C04600C09FE5D0
:101750001CFF2FE14D8000C07847C04600C09FE5C8
:101760001CFF2FE15D8000C01D2E04EA282E04EA34
:10177000E22D04EADB0F04EA091104EAD70F04EAB8
:10178000C62E04EA7847C04600C09FE51CFF2FE143
:1017900071D400C0B52E04EA462004EAA32004EA6E
:1017A000422004EA7847C04600C09FE51CFF2FE1B5
:1017B000B18600C07847C04600C09FE51CFF2FE1FE
:1017C000AD8700C07847C04600C09FE51CFF2FE1F1
:1017D000CD7F00C07847C04600C09FE51CFF2FE1C9
:1017E00081AE00C07847C04600C09FE51CFF2FE1D6
:1017F000D9AE00C0AB2504EA7847C04600C09FE5DB
:101800001CFF2FE1691B01C07847C04600C09FE55F
:101810001CFF2FE1991D01C07847C04600C09FE51D
:101820001CFF2FE13F1901C08D3204EAB73204EAF0
:10183000613204EA941804EA951804EA901804EA5C
:101840007847C04600C09FE51CFF2FE1E94EF0BF7E
:101850007847C04600C09FE51CFF2FE14D3401C012
:101860007847C04600C09FE51CFF2FE1AD2C01C0AA
:101870007847C04600C09FE51CFF2FE1652101C0ED
:101880007847C04600C09FE51CFF2FE1B52101C08D
:101890007847C04600C09FE51CFF2FE1512101C0E1
:1018A0007847C04600C09FE51CFF2FE1851901C0A5
:1018B0007847C04600C09FE51CFF2FE1DF1A01C03A
:1018C0007847C04600C09FE51CFF2FE1291B01C0DF
:1018D0007847C04600C09FE51CFF2FE1211A01C0D8
:1018E000AD2305EA471A05EA896304EAB26A04EA05
:1018F000E36804EA4B1A05EA3C0F00EA556304EA80
:10190000767804EACB7304EA697104EA366304EA80
:10191000496104EA366204EA816304EA627805EA0E
:1019200017FF04EA2C7505EAF96204EAE0FC04EA10
:10193000C09304EADF0E00EA00C09FE51CFF2FE120
:101940001D8E05C0B51C04EA082604EA00C09FE508
:101950001CFF2FE1D1D504C0CC4904EA00C09FE5AB
:101960001CFF2FE1156F03C0172E04EA00C09FE58E
:101970001CFF2FE18DD205C000C09FE51CFF2FE1A9
:10198000B10405C0EF0700EA00C09FE51CFF2FE18E
:10199000F19D03C07847C04600C09FE51CFF2FE1C2
:1019A00039D005C07847C04600C09FE51CFF2FE135
:1019B0005D0205C07847C04600C09FE51CFF2FE1CF
:1019C0009D9B03C0E97305EAE2E704EA4F7704EA66
:1019D000862405EA008B04EA449204EA8D6A04EA4C
:1019E000736204EA496204EA7A7104EAB1B804EA6B
:1019F000C09304EA27B904EADAE904EAE29804EABF
:101A0000542205EA4A4105EAB3E404EADEB804EAEE
:101A1000C27804EA2C9804EA80E904EABB9204EA5A
:101A200058A504EAE9B604EA1B2C05EA6DD204EADB
:101A300005A304EADEA204EAD27804EAF07804EA14
:101A40008A2505EA5FB704EA59EA04EA5CB604EAC3
:101A50008DE904EA337505EAD18604EA388C04EA94
:101A6000138704EA248C04EA7C8B04EABA9104EA22
:101A7000309104EA369104EA236204EA5F7704EACB
:101A8000DD6E04EA417704EA148504EAE27404EAAC
:101A9000427104EA5B9104EA2F9104EAD39104EACB
:101AA0009F8E04EA0D8E04EAD28C04EA738C04EA59
:101AB0003B8D04EA248D04EA608E04EAB5F104EA61
:101AC00071F904EA369804EAF18B04EA4F8D04EACE
:101AD000A98804EA519104EA162705EAFE8B04EA74
:101AE00053A304EAD5C504EAD6C504EAE3E804EA48
:101AF00023E904EA906804EADE7404EA4D7804EA13
:101B0000247504EA806804EA636804EA196004EA58
:101B1000B16E05EACCA304EA5B7205EA7DAF04EA84
:101B200065E604EA244205EA5DC004EAAD5505EA2B
:101B3000484C05EA20A804EA59D204EA052C05EA33
:101B4000D79B04EAF4BB04EACEC204EA3A8204EA70
:101B5000F3C704EADFB004EA3CA304EAA7BF04EA3F
:101B6000ED9804EAE4B604EA702305EA7847C04633
:101B700000C09FE51CFF2FE1954703C07847C04692
:101B800000C09FE51CFF2FE1C14703C07847C04656
:101B900000C09FE51CFF2FE1794803C07847C0468D
:101BA00000C09FE51CFF2FE1454A03C07847C046AF
:101BB00000C09FE51CFF2FE16F7F03C07847C04640
:101BC00000C09FE51CFF2FE1ED4A03C07847C046E7
:101BD00000C09FE51CFF2FE1814C03C07847C04641
:101BE00000C09FE51CFF2FE1494703C07847C0466E
:101BF00000C09FE51CFF2FE1D94C03C07847C046C9
:101C000000C09FE51CFF2FE1254B03C07847C0466D
:101C100000C09FE51CFF2FE1477F03C07847C04607
:101C200000C09FE51CFF2FE1414F03C07847C0462D
:101C300000C09FE51CFF2FE16D4F03C07847C046F1
:101C400000C09FE51CFF2FE1255003C07847C04628
:101C500000C09FE51CFF2FE1F15103C07847C0464B
:101C600000C09FE51CFF2FE12BE604C07847C0466B
:101C700000C09FE51CFF2FE1995203C07847C04682
:101C800000C09FE51CFF2FE12D5403C07847C046DC
:101C900000C09FE51CFF2FE1F54E03C07847C0460A
:101CA00000C09FE51CFF2FE1855403C07847C04664
:101CB00000C09FE51CFF2FE1D15203C07847C0460A
:101CC00000C09FE51CFF2FE103E604C07847C04633
:101CD00000C09FE51CFF2FE11D6D03C07847C04683
:101CE00000C09FE51CFF2FE1316B03C07847C04661
:101CF00000C09FE51CFF2FE1716E03C07847C0460E
:101D000000C09FE51CFF2FE1156A03C07847C0465D
:101D100000C09FE51CFF2FE1659A03C07847C046CD
:101D200000C09FE51CFF2FE1896D03C07847C046C6
:101D300000C09FE51CFF2FE1CD6E03C07847C04671
:101D400000C09FE51CFF2FE1516F03C07847C046DC
:101D500000C09FE51CFF2FE1599B03C07847C04698
:101D600000C09FE51CFF2FE1018203C07847C046F9
:101D700000C09FE51CFF2FE1E59A03C07847C046ED
:101D800000C09FE51CFF2FE1996F03C07847C04654
:101D900000C09FE51CFF2FE1317003C07847C046AB
:101DA00000C09FE51CFF2FE1FD7603C07847C046C9
:101DB00000C09FE51CFF2FE1257103C07847C04696
:101DC00000C09FE51CFF2FE1317F03C07847C0466C
:101DD00000C09FE51CFF2FE1117303C07847C04688
:101DE00000C09FE51CFF2FE1A97B03C07847C046D8
:101DF00000C09FE51CFF2FE1997C03C07847C046D7
:101E000000C09FE51CFF2FE1359703C07847C0460F
:101E100000C09FE51CFF2FE19D8203C07847C046AC
:101E200000C09FE51CFF2FE1D56703C07847C0467F
:101E300000C09FE51CFF2FE1218103C07847C04609
:101E400000C09FE51CFF2FE1398103C07847C046E1
:101E500000C09FE51CFF2FE1E17F03C07847C0462B
:101E600000C09FE51CFF2FE1917F03C07847C0466B
:101E700000C09FE51CFF2FE1B18003C07847C0463A
:101E800000C09FE51CFF2FE10D4D03C07847C04601
:101E900000C09FE51CFF2FE1D14B03C07847C0462F
:101EA00000C09FE51CFF2FE15D8003C07847C0465E
:101EB00000C09FE51CFF2FE1498103C07847C04661
:101EC00000C09FE51CFF2FE11D6F03C07847C0468F
:101ED00000C09FE51CFF2FE1458A03C07847C0463C
:101EE00000C09FE51CFF2FE1218903C07847C04651
:101EF00000C09FE51CFF2FE1B99603C07847C0469C
:101F000000C09FE51CFF2FE1F98F03C07847C04652
:101F100000C09FE51CFF2FE1399503C07847C046FC
:101F200000C09FE51CFF2FE16D9503C07847C046B8
:101F300000C09FE51CFF2FE1E17C03C07847C0464D
:101F400000C09FE51CFF2FE1B17103C07847C04678
:101F500000C09FE51CFF2FE16D7E03C07847C0469F
:101F600000C09FE51CFF2FE1F17B03C07847C0460E
:101F700000C09FE51CFF2FE1AF7C03C07847C0463F
:101F800000C09FE51CFF2FE1C58703C07847C0460E
:101F900000C09FE51CFF2FE1B19503C07847C04604
:101FA00000C09FE51CFF2FE1299A03C07847C04677
:101FB00000C09FE51CFF2FE18D9503C07847C04608
:101FC00000C09FE51CFF2FE1DD7D03C07847C046C0
:101FD00000C09FE51CFF2FE1597203C07847C0463F
:101FE00000C09FE51CFF2FE1C59503C07847C046A0
:101FF000300D00EA7847C04600C09FE51CFF2FE186
:10200000DD7A03C07847C04600C09FE51CFF2FE182
:10201000E59603C07847C04600C09FE51CFF2FE14E
:10202000619603C07847C04600C09FE51CFF2FE1C2
:10203000259A03C07847C04600C09FE51CFF2FE1EA
:10204000319103C07847C04600C09FE51CFF2FE1D7
:10205000C97F03C07847C04600C09FE51CFF2FE141
:10206000259B03C07847C04600C09FE51CFF2FE1B9
:10207000199603C07847C04600C09FE51CFF2FE1BA
:10208000A98103C07847C04600C09FE51CFF2FE12F
:102090008D8F03C07847C04600C09FE51CFF2FE12D
:1020A000D99703C07847C04600C09FE51CFF2FE1C9
:1020B000839503C07847C046B99604EA7847C0467E
:1020C00000C09FE51CFF2FE19D8B03C07847C046F1
:1020D00000C09FE51CFF2FE1319E03C07847C0463A
:1020E00000C09FE51CFF2FE17D9803C07847C046E4
:1020F00000C09FE51CFF2FE19D9703C07847C046B5
:1021000000C09FE51CFF2FE14D8903C07847C04602
:1021100000C09FE51CFF2FE1B19103C07847C04686
:1021200000C09FE51CFF2FE1CD8803C07847C04663
:1021300000C09FE51CFF2FE1AD9303C07847C04668
:1021400000C09FE51CFF2FE10D8A03C07847C04601
:1021500000C09FE51CFF2FE1DD8903C07847C04622
:1021600000C09FE51CFF2FE1A98603C07847C04649
:1021700000C09FE51CFF2FE15D9403C07847C04677
:1021800000C09FE51CFF2FE1B19403C07847C04613
:1021900000C09FE51CFF2FE1619303C07847C04654
:1021A00000C09FE51CFF2FE1218603C07847C04691
:1021B00000C09FE51CFF2FE1E99303C07847C046AC
:1021C00000C09FE51CFF2FE1399203C07847C0464D
:1021D00000C09FE51CFF2FE15D9603C07847C04615
:1021E00000C09FE51CFF2FE14D9103C07847C0461A
:1021F00000C09FE51CFF2FE1E98203C07847C0467D
:1022000000C09FE51CFF2FE1518503C07847C04601
:1022100000C09FE51CFF2FE1E78803C07847C04658
:1022200000C09FE51CFF2FE1098C03C07847C04622
:1022300000C09FE51CFF2FE1A18B03C07847C0467B
:1022400000C09FE51CFF2FE1158E03C07847C046F4
:1022500000C09FE51CFF2FE1159403C0C9E304EA09
:10226000139604EA0CFD04EA4C2605EA1D2305EA50
:1022700054E804EA54EB04EA84EC04EA29F104EAA1
:10228000AAED04EAF4EE04EA84F004EA46EF04EA74
:1022900061F004EA7DEF04EAA3F004EA37F004EA0F
:1022A000C4F904EA9FF304EAD6F104EAFAF104EA75
:1022B0000AEE04EAD5F204EA0CF604EA46F504EA6A
:1022C000B5F204EA6CF104EA20F204EAD4EE04EA7E
:1022D000F3F604EAEBEE04EA6AF704EAC2F404EA6D
:1022E0002DFA04EA25FA04EAF4EE04EA677604EA31
:1022F000970C00EA002105EA0F4205EAF02405EAFE
:10230000449104EA6B2105EACFE504EACEC304EA6E
:10231000664605EAC34605EA8A4605EA202105EA3B
:10232000AD7604EAE21A05EA6D9A04EA85FD04EA4C
:10233000FA6C05EA5A4B05EA103C05EA7ADF04EA32
:10234000EB9D04EACBAA04EACDBA04EA10C204EA7F
:1023500009C704EAE48004EAEAAF04EA609B04EAFD
:10236000F9C004EA94A704EA2FE804EA1E3905EA52
:10237000791205EA3F6D04EAC36404EAC26C04EA18
:10238000336F04EA786204EAFD6004EAC21F05EADA
:102390001BA704EA272105EAA36C04EA9CAE04EA21
:1023A000029304EA929204EA769104EAF99104EA2B
:1023B000179304EAC49104EACB2705EA8CB504EA32
:1023C000C9E504EA874805EA8DA404EA7BCE04EA5D
:1023D000272805EA4D9804EA49B804EAAC7E04EAE5
:1023E000BB5105EADD4605EA01A304EACACC04EACA
:1023F000162605EADD9604EAABB604EA0BBF04EA4A
:102400003BC404EA367D04EAEC4F05EA527005EA63
:10241000F34E05EAB0AD04EA4CE404EA0B4005EAE9
:10242000A19F04EA43BE04EA09C304EAEDC504EA35
:10243000418104EAFAB204EAEC9C04EA817604EAF7
:10244000889004EABD9004EA9D4105EAAC4105EAA2
:10245000528204EA8F1705EA9F1A05EA690205EA23
:102460003D2105EA31A104EAC07505EA7847C04676
:1024700000C09FE51CFF2FE1D1D304C07847C046C0
:1024800000C09FE51CFF2FE1E5D104C07847C0469E
:1024900000C09FE51CFF2FE12DD504C07847C04642
:1024A00000C09FE51CFF2FE1C9D004C07847C0469B
:1024B00000C09FE51CFF2FE1250105C07847C046FD
:1024C00000C09FE51CFF2FE13DD404C07847C04603
:1024D00000C09FE51CFF2FE189D504C07847C046A6
:1024E00000C09FE51CFF2FE10DD604C07847C04611
:1024F00000C09FE51CFF2FE1190205C07847C046C8
:1025000000C09FE51CFF2FE1BDE804C07847C0462E
:1025100000C09FE51CFF2FE1A50105C07847C0461C
:1025200000C09FE51CFF2FE155D604C07847C04688
:1025300000C09FE51CFF2FE1EDD604C07847C046E0
:1025400000C09FE51CFF2FE1B9DD04C07847C046FD
:1025500000C09FE51CFF2FE1E1D704C07847C046CB
:1025600000C09FE51CFF2FE1EDE504C07847C046A1
:1025700000C09FE51CFF2FE1CDD904C07847C046BD
:1025800000C09FE51CFF2FE165E204C07847C0460C
:1025900000C09FE51CFF2FE155E304C07847C0460B
:1025A00000C09FE51CFF2FE1F5FD04C07847C04641
:1025B00000C09FE51CFF2FE159E904C07847C046E1
:1025C00000C09FE51CFF2FE189CE04C07847C046BC
:1025D00000C09FE51CFF2FE1DDE704C07847C0463F
:1025E00000C09FE51CFF2FE1F5E704C07847C04617
:1025F00000C09FE51CFF2FE19DE604C07847C04660
:1026000000C09FE51CFF2FE14DE604C07847C0469F
:1026100000C09FE51CFF2FE16DE704C07847C0466E
:1026200000C09FE51CFF2FE1B95403C07847C046A6
:1026300000C09FE51CFF2FE17D5303C07847C046D3
:1026400000C09FE51CFF2FE119E704C07847C04692
:1026500000C09FE51CFF2FE105E804C07847C04695
:1026600000C09FE51CFF2FE1D9D504C07847C046C4
:1026700000C09FE51CFF2FE101F104C07847C04670
:1026800000C09FE51CFF2FE1DDEF04C07847C04686
:1026900000C09FE51CFF2FE179FD04C07847C046CC
:1026A00000C09FE51CFF2FE1B5F604C07847C04687
:1026B00000C09FE51CFF2FE1F9FB04C07847C0462E
:1026C00000C09FE51CFF2FE12DFC04C07847C046E9
:1026D00000C09FE51CFF2FE19DE304C07847C04682
:1026E00000C09FE51CFF2FE16DD804C07847C046AD
:1026F00000C09FE51CFF2FE129E504C07847C046D4
:1027000000C09FE51CFF2FE1ADE204C07847C04642
:1027100000C09FE51CFF2FE16BE304C07847C04673
:1027200000C09FE51CFF2FE181EE04C07847C04642
:1027300000C09FE51CFF2FE171FC04C07847C04634
:1027400000C09FE51CFF2FE1E90005C07847C046A7
:1027500000C09FE51CFF2FE14DFC04C07847C04638
:1027600000C09FE51CFF2FE199E404C07847C046F4
:1027700000C09FE51CFF2FE115D904C07847C04673
:1027800000C09FE51CFF2FE185FC04C07847C046D0
:1027900000C09FE51CFF2FE199E104C07847C046C7
:1027A00000C09FE51CFF2FE1A5FD04C07847C0468F
:1027B00000C09FE51CFF2FE121FD04C07847C04603
:1027C00000C09FE51CFF2FE1E50005C07847C0462B
:1027D00000C09FE51CFF2FE1EDF704C07847C0461D
:1027E00000C09FE51CFF2FE185E604C07847C04686
:1027F00000C09FE51CFF2FE1E50105C07847C046FA
:1028000000C09FE51CFF2FE1D9FC04C07847C046FB
:1028100000C09FE51CFF2FE165E804C07847C04673
:1028200000C09FE51CFF2FE149F604C07847C04671
:1028300000C09FE51CFF2FE199FE04C07847C04609
:1028400000C09FE51CFF2FE143FC04C07847C04651
:1028500000C09FE51CFF2FE159F204C07847C04635
:1028600000C09FE51CFF2FE1F10405C07847C0467A
:1028700000C09FE51CFF2FE13DFF04C07847C04624
:1028800000C09FE51CFF2FE15DFE04C07847C046F5
:1028900000C09FE51CFF2FE109F004C07847C04647
:1028A00000C09FE51CFF2FE171F804C07847C046C7
:1028B00000C09FE51CFF2FE189EF04C07847C046A8
:1028C00000C09FE51CFF2FE16DFA04C07847C046A9
:1028D00000C09FE51CFF2FE1C9F004C07847C04647
:1028E00000C09FE51CFF2FE199F004C07847C04667
:1028F00000C09FE51CFF2FE165ED04C07847C0468E
:1029000000C09FE51CFF2FE11DFB04C07847C046B7
:1029100000C09FE51CFF2FE171FB04C07847C04653
:1029200000C09FE51CFF2FE121FA04C07847C04694
:1029300000C09FE51CFF2FE1DDEC04C07847C046D6
:1029400000C09FE51CFF2FE1A9FA04C07847C046EC
:1029500000C09FE51CFF2FE1F9F804C07847C0468E
:1029600000C09FE51CFF2FE11DFD04C07847C04655
:1029700000C09FE51CFF2FE109F804C07847C0465E
:1029800000C09FE51CFF2FE1A5E904C07847C046C1
:1029900000C09FE51CFF2FE10DEC04C07847C04646
:1029A00000C09FE51CFF2FE1A3EF04C07847C0469D
:1029B00000C09FE51CFF2FE1C5F204C07847C04668
:1029C00000C09FE51CFF2FE15DF204C07847C046C0
:1029D00000C09FE51CFF2FE1D1F404C07847C0463A
:1029E00000C09FE51CFF2FE1D5FA04C0A39304EAC1
:1029F000593F05EAF5E304EA18E404EA710005EA40
:102A0000DB8E04EA3A2405EA7847C04600C09FE519
:102A10001CFF2FE1457B05C07847C04600C09FE5FD
:102A20001CFF2FE11F7A05C07847C04600C09FE514
:102A30001CFF2FE1957B05C07847C04600C09FE58D
:102A40001CFF2FE1AD7B05C07847C04600C09FE565
:102A50001CFF2FE17D7B05C07847C04600C09FE585
:102A60001CFF2FE1B97805C07847C04600C09FE53C
:102A70001CFF2FE131A305C07847C04600C09FE589
:102A80001CFF2FE119A305C07847C04600C09FE591
:102A90001CFF2FE1E97F05C07847C04600C09FE5D5
:102AA0001CFF2FE1C57B05C07847C04600C09FE5ED
:102AB0001CFF2FE1D9CB05C07847C04600C09FE579
:102AC0001CFF2FE115CC05C07847C04600C09FE52C
:102AD0001CFF2FE1DDCC05C07847C04600C09FE554
:102AE0001CFF2FE15DCD05C07847C04600C09FE5C3
:102AF0001CFF2FE111CF05C07847C04600C09FE5FD
:102B00001CFF2FE18DCD05C07847C04600C09FE572
:102B10001CFF2FE16F8105C07847C04600C09FE5CC
:102B20001CFF2FE1197905C07847C04600C09FE51A
:102B30001CFF2FE1597A05C07847C04600C09FE5C9
:102B40001CFF2FE1817905C07847C04600C09FE592
:102B50001CFF2FE15D8705C07847C04600C09FE598
:102B60001CFF2FE1718505C07847C04600C09FE576
:102B70001CFF2FE1F1A505C07847C04600C09FE5C6
:102B80001CFF2FE1B98805C07847C04600C09FE50B
:102B90001CFF2FE1F18905C07847C04600C09FE5C2
:102BA0001CFF2FE1398405C07847C04600C09FE56F
:102BB0001CFF2FE1C5C605C07847C04600C09FE591
:102BC0001CFF2FE1C98705C07847C04600C09FE5BC
:102BD0001CFF2FE1158905C07847C0462B7404EA15
:102BE0007847C0460C4405EA7847C04600C09FE5D8
:102BF0001CFF2FE1598E05C07847C04600C09FE5F5
:102C00001CFF2FE1B9C705C07847C04600C09FE54B
:102C10001CFF2FE189A405C07847C04600C09FE58E
:102C20001CFF2FE145C705C07847C04600C09FE59F
:102C30001CFF2FE1A18E05C07847C04600C09FE56C
:102C40001CFF2FE1599305C07847C04600C09FE59F
:102C50001CFF2FE16D8F05C07847C04600C09FE57F
:102C60001CFF2FE15D9C05C07847C04600C09FE572
:102C70001CFF2FE1D99105C07847C04600C09FE5F1
:102C80001CFF2FE1C99805C07847C04600C09FE5EA
:102C90001CFF2FE10D8F05C07847C04600C09FE59F
:102CA0001CFF2FE1C99905C07847C04600C09FE5C9
:102CB0001CFF2FE179C305C07847C04600C09FE5DF
:102CC0001CFF2FE141A505C07847C04600C09FE525
:102CD0001CFF2FE1DFC205C07847C04600C09FE55A
:102CE0001CFF2FE1337A05C07847C04600C09FE53E
:102CF0001CFF2FE1C9C805C07847C04600C09FE54A
:102D00001CFF2FE1D7CB05C07847C04600C09FE528
:102D10001CFF2FE10DA005C07847C04600C09FE50D
:102D20001CFF2FE17DA205C07847C04600C09FE58B
:102D30001CFF2FE1AD9E05C07847C04600C09FE54F
:102D40001CFF2FE1759C05C07847C04600C09FE579
:102D50001CFF2FE141A305C07847C04600C09FE596
:102D60001CFF2FE17D9D05C07847C04600C09FE550
:102D70001CFF2FE105A405C07847C04600C09FE5B1
:102D80001CFF2FE11D7505C07847C04600C09FE5B8
:102D90001CFF2FE1598005C07847C04600C09FE561
:102DA0001CFF2FE1B59D05C07847C04600C09FE5D8
:102DB0001CFF2FE1197D05C07847C04600C09FE584
:102DC0001CFF2FE1B97505C07847C04600C09FE5DC
:102DD0001CFF2FE1258E05C07847C04600C09FE547
:102DE0001CFF2FE18DA505C07847C04600C09FE5B8
:102DF0001CFF2FE155C105C07847C04600C09FE5C4
:102E00001CFF2FE189C605C07847C04600C09FE57A
:102E10001CFF2FE18DAF05C07847C04600C09FE57D
:102E20001CFF2FE1FFC205C07847C04600C09FE5E8
:102E30001CFF2FE145BA05C07847C04600C09FE59A
:102E40001CFF2FE111C105C07847C04600C09FE5B7
:102E50001CFF2FE141B105C07847C04600C09FE587
:102E60001CFF2FE175C005C07847C04600C09FE534
:102E70001CFF2FE1119A05C07847C04600C09FE5AE
:102E80001CFF2FE10D9005C07847C04600C09FE5AC
:102E90001CFF2FE19D9B05C07847C04600C09FE501
:102EA0001CFF2FE11D9905C07847C04600C09FE573
:102EB0001CFF2FE1DF9905C07847C04600C09FE5A1
:102EC0001CFF2FE199AD05C07847C04600C09FE5C3
:102ED0001CFF2FE131C105C07847C04600C09FE507
:102EE0001CFF2FE10D9B05C07847C04600C09FE541
:102EF0001CFF2FE1B59205C07847C04600C09FE592
:102F00001CFF2FE169C105C07847C04600C09FE59E
:102F10001CFF2FE19D8105C07847C04600C09FE59A
:102F20001CFF2FE1BDAE05C07847C04600C09FE53D
:102F30001CFF2FE1B96905C07847C04600C09FE576
:102F40001CFF2FE199BB05C07847C04600C09FE534
:102F50001CFF2FE1FD9705C07847C04600C09FE5E4
:102F60001CFF2FE129C305C07847C04600C09FE57C
:102F70001CFF2FE13DC605C07847C04600C09FE555
:102F80001CFF2FE165C205C07847C04600C09FE521
:102F90001CFF2FE17DBB05C07847C04600C09FE500
:102FA0001CFF2FE1359E05C07847C04600C09FE555
:102FB0001CFF2FE185C705C07847C04600C09FE5CC
:102FC0001CFF2FE1BDC105C07847C04600C09FE58A
:102FD0001CFF2FE1B9AF05C07847C04600C09FE590
:102FE0001CFF2FE109A405C07847C04600C09FE53B
:102FF0001CFF2FE1D9B905C07847C04600C09FE546
:103000001CFF2FE11DC405C07847C04600C09FE5E6
:103010001CFF2FE127C105C07847C04600C09FE5CF
:103020001CFF2FE1F9C705C07847C04600C09FE5E7
:103030001CFF2FE1ED6905C07847C04600C09FE541
:103040001CFF2FE1ADCB05C07847C04600C09FE50F
:103050001CFF2FE199B205C07847C04600C09FE52C
:103060001CFF2FE1D5D205C07847C04600C09FE5C0
:103070001CFF2FE1C1C405C07847C04600C09FE5D2
:103080001CFF2FE1E1C305C07847C04600C09FE5A3
:103090001CFF2FE1E1CA05C07847C04600C09FE58C
:1030A0001CFF2FE14DB005C07847C04600C09FE52A
:1030B0001CFF2FE199BC05C07847C04600C09FE5C2
:1030C0001CFF2FE1A1AE05C07847C04600C09FE5B8
:1030D0001CFF2FE1E9BE05C07847C04600C09FE550
:1030E0001CFF2FE109B105C07847C04600C09FE52D
:1030F0001CFF2FE1D9B005C07847C04600C09FE54E
:103100001CFF2FE17DAC05C07847C04600C09FE59D
:103110001CFF2FE199BF05C07847C04600C09FE55E
:103120001CFF2FE1EDBF05C07847C04600C09FE5FA
:103130001CFF2FE19DBE05C07847C04600C09FE53B
:103140001CFF2FE1F5AB05C07847C04600C09FE5E6
:103150001CFF2FE125BF05C07847C04600C09FE592
:103160001CFF2FE141BD05C07847C04600C09FE568
:103170001CFF2FE101C205C07847C04600C09FE593
:103180001CFF2FE1B1A705C07847C04600C09FE5EE
:103190001CFF2FE135BC05C07847C04600C09FE545
:1031A0001CFF2FE1E9A805C07847C04600C09FE595
:1031B0001CFF2FE125AB05C07847C04600C09FE546
:1031C0001CFF2FE151AF05C07847C04600C09FE506
:1031D0001CFF2FE1F9B505C07847C04600C09FE548
:1031E0001CFF2FE191B505C07847C04600C09FE5A0
:1031F0001CFF2FE155B805C07847C04600C09FE5C9
:103200001CFF2FE151BF05C0707E04EA376404EA59
:10321000B43E05EAFA6804EA876604EA601C05EA37
:103220009EB004EA956404EAD38404EA928104EA35
:10323000C18304EA458004EADE8304EAB58504EA32
:10324000098604EA408204EAFA8004EAF48304EA84
:10325000C18104EA468304EA078504EAAE8404EAED
:10326000408504EAD18304EA018504EA838004EA04
:103270009C8504EA698404EA648104EA108204EA11
:103280006D8504EA4C8004EA418004EA278504EA5B
:103290008A8104EA428104EA138404EA776204EA38
:1032A000676204EA2DEB04EAAAF504EA85F504EA6C
:1032B0007FED04EAB1EA04EAB3EC04EA63F604EA57
:1032C00088EA04EA7847C04600C09FE51CFF2FE16A
:1032D0008DD205C07847C04600C09FE51CFF2FE196
:1032E00035D005C07847C04600C09FE51CFF2FE1E0
:1032F000B10405C07847C04600C09FE51CFF2FE120
:10330000590205C07847C04600C09FE51CFF2FE169
:10331000F19D03C07847C04600C09FE51CFF2FE128
:10332000999B03C0770D07EA960D07EA7D0D07EA22
:10333000630D07EA750D07EAB40F07EA770E07EA8F
:10334000D60D07EA130F07EAC60E07EA260E07EAAC
:10335000620F07EA0F1007EA001007EA7D1007EA7C
:10336000531007EA111107EA661007EA8A1007EA04
:10337000C61007EA400D07EAFD1007EA2C1007EA1D
:10338000BC0F07EAD70F07EA00000000E07D0CC081
:10339000FC7F0C000300000007000000000000009C
:1033A000000000000300000000000000000000001A
:1033B00044010000000000000000000007000000C1
:1033C00001000000010000000000000000000000FB
:1033D00000000000000000000000000003000000EA
:1033E00007000000000000000000000003000000D3
:1033F00000000000000000001B00000000000000B2
:1034000000000000070000000100000000000000B4
:1034100000000000000000000000000000000000AC
:103420000000000003000000070000000000000092
:103430000000000003000000000000000000000089
:10344000070000000000000000000000070000006E
:10345000000000000100000000000000000000006B
:10346000000000000000000000000000020000005A
:103470000700000001000000010000000000000043
:103480000000000000000000060000000100000035
:103490000000000007000000000000000000000025
:1034A000000000000000000000000000000000001C
:1034B0000000000061D3083200000000000000009E
:1034C00000000000CE0C0000CE0C00000A0000003E
:1034D0001F000000000000000000000001000000CC
:1034E00005000000A4000000000000007C000E00A9
:1034F00005010000000000000000000000000000C6
:103500005F5F444154455F5F205F5F54494D455FB5
:103510005F00000002000000010000000600000043
:103520008434F0BF00000000000000000000000034
:10353000000000000000000000000000000000008B
:10354000000100000000000000000000000000007A
:103550000000000000000000020000000000000069
:103560000000010000000100010000000B006600E7
:10357000C434F0BF20000000000000000B00670012
:103580000000000002000000010000000B006800C5
:10359000E434F0BF02000000000000000B006900EE
:1035A0000000000006000000FFFFFFFF0000000019
:1035B0000000000000000000010000000B006A0095
:1035C000EA34F0BF02000000000000000B006B00B6
:1035D0000000000002000000FFFFFFFF00000000ED
:1035E0000000000000000000010000000B006C0063
:1035F000E634F0BF02000000000000000B006D0088
:103600000000000004000000FFFFFFFF00000000BA
:103610000000000000000000010000000B006C0032
:10362000E834F0BF02000000000000000B006D0055
:103630000000000004000000FFFFFFFF000000008A
:10364000000000000000000000000000000000007A
:10365000000000000000000000000000000000006A
:1036600000000000000000005C02F0BF000000004D
:1036700000000000149701C00000000000000000DE
:10368000000000000000000000000000000000003A
:10369000000000000000000000000000000000002A
:1036A000000000000000000000000000000000001A
:1036B000000000000000000000000000000000000A
:10394000000000000000000070402DE9045090E5E8
:103950000040A0E10500A0E1F11EA0E3F4F7FFEBB9
:103960000400A0E1045084E559F8FFEB0400A0E155
:1039700059F8FFEB7040BDE80000A0E31EFF2FE107
:10398000A4FC03EA7847C04600C09FE51CFF2FE176
:10399000BB2800C07847C046DCFB03EA1DFB03EAF6
:1039A0007847C04600C09FE51CFF2FE1C92300C037
:1039B0007847C046D60400EA6C009FE510402DE928
:1039C000280090E5020C10E30900A0130200001A81
:1039D000010B10E30300000A0A00A0E352F2FFEB20
:1039E0001040BDE81EFF2FE1010C10E30300000AA8
:1039F0000800A0E34DF2FFEB1040BDE81EFF2FE1F1
:103A0000020010E30300000A0100A0E348F2FFEB0C
:103A10001040BDE81EFF2FE1010010E30000A013DD
:103A200044F2FF1B1040BDE81EFF2FE1000300F829
:103A3000FE432DE90170A0E19C12D0E50280A0E1D7
:103A40009D22D0E50360A0E10030A0E30E008DE8E8
:103A50000050A0E10400D6E50020D6E50310D6E52D
:103A600038F2FFEB0040B0E12700001A0630A0E179
:103A70000820A0E10710A0E10500A0E13BF2FFEB68
:103A80000040B0E12000001A0400D6E5020050E337
:103A90001500001A9C12D5E59D22D5E50030A0E363
:103AA0000E008DE80020D6E50310D6E52500D5E50B
:103AB0000130A0E323F2FFEB0040B0E11200001A56
:103AC0000320D6E52810D5E50500A0E120F2FFEBA4
:103AD0000040B0E10C00001A0500A0E1690000EB15
:103AE0000048A0E12448A0E1070000EA380095E57D
:103AF000000050E3F1FFFF1A0500A0E12D0000EBEC
:103B00000040A0E10500A0E11BF2FFEB0430A0E1C2
:103B10000620A0E10B10A0E30700A0E10EF2FFEBEE
:103B2000FE43BDE81EFF2FE130402DE914D04DE2E9
:103B30000050A0E30040A0E108508DE5740090E53E
:103B4000000050E30110A0130400A011745084156C
:103B50000BF2FF1B700094E5000050E370508415D9
:103B6000020000EA10109DE50400A0E105F2FFEB61
:103B700004308DE200308DE50C308DE208208DE2BE
:103B800010108DE2900084E2FFF1FFEB000050E3A3
:103B9000F3FFFF0A0800DDE5000050E36C209415F8
:103BA000BA16D4110400A011EEF1FF1B14D08DE25F
:103BB0003040BDE81EFF2FE170402DE90040A0E13C
:103BC0000C0090E50050A0E3000050E30F00000A55
:103BD000380094E5000050E30C00001A0000A0E358
:103BE0003B0200EB900084E2ECF1FFEB000050E3BD
:103BF0000000A0E30C0084E51C509F15200084E524
:103C00000200001A6400D4E5E5F1FFEB0050A0E1EA
:103C10000500A0E17040BDE81EFF2FE161800000BB
:103C200070402DE958509FE50040A0E3000095E565
:103C3000900080E2DFF1FFEB030010E30010951528
:103C40000120A0E30140A01370208115200010E3A3
:103C50000400000A000095E50010D0E5020051E3E1
:103C600074208005010000EA000054E30100000A0E
:103C70000100A0E3D0F1FFEB7040BDE80100A0E33C
:103C80001EFF2FE1C034F0BF70402DE90050A0E3CB
:103C90000040A0E1205080E50C0090E5000050E3DA
:103CA0001600001A0020A0E33010E0E30400A0E1B9
:103CB000CEF1FFEB0400A0E33401C4E5900084E200
:103CC000CDF1FFEB0050B0E10300001A6400D4E531
:103CD000B3F1FFEB000050E31600001A0100A0E36F
:103CE0000C0084E5100094E5000050E3F418D401C2
:103CF0000120A0030400A001BCF1FF0B090000EAB1
:103D0000010050E30700001A380094E5000050E37A
:103D10000400000A24009FE5000090E5900080E286
:103D2000A4F1FFEB1D5000E20100A0E3E80100EB6D
:103D30000500B0E108009F157040BDE81EFF2FE1AF
:103D4000C034F0BF6180000070402DE90150A0E157
:103D50000B0052E30210A0E10360A0E10040A0E1EB
:103D60001500000A0D0051E31700000A110051E38D
:103D70001100000A860051E31800001A0610A0E1A5
:103D80000400A0E1B0F1FFEB2700D4E5020050E30E
:103D9000000050130400001A0400A0E1B9FFFFEB7B
:103DA000000050E348009F1563F1FF1B0200A0E3F1
:103DB0000000C4E57040BDE81EFF2FE134309FE5F0
:103DC0000620A0E10500A0E163F1FFEB0620A0E1E1
:103DD0000510A0E10400A0E19CF1FFEBF4FFFFEA75
:103DE00014309FE50620A0E10500A0E15AF1FFEBA9
:103DF000EFFFFFEA61800000224000002640000043
:103E000010402DE90100A0E394F1FFEB0100A0E3D5
:103E100093F1FFEB1040BDE81EFF2FE1F8B5040061
:103E200088682121008809026518002716000028EB
:103E300001D01B4E00E0EF701A48201846801A4847
:103E40002018007C00280AD0012825D128780028D5
:103E500003D1FFF7ADFD002805D1277307E020004F
:103E6000FCF782FB17E01149012020734870200005
:103E7000FCF782FB0C49200084398030FCF784FB7E
:103E8000832080012018476387636878002803D166
:103E90002000FCF781FB06003000F8BC08BC184786
:103EA0000C41000060310000E0200000E079F0BF2C
:103EB000F8B50400886821210088090266180028E6
:103EC00001D0274A01E00120F07026482018028026
:103ED0002448283021182000002300F04BFA050068
:103EE00021480021017021482718797C08002843C7
:103EF00003D12000FCF760FB0500787C012805D188
:103F0000002D08D12000FCF75FFB0500002D02D139
:103F1000042020731FE0387C002806D001281AD125
:103F20003078002806D0002005E02000FCF71CFBBC
:103F3000050010E0012020732000FCF71DFB0B4959
:103F4000200084398030FCF71FFB83218901002089
:103F50006118486388632800F8BC08BC1847000053
:103F60000B41000060310000E079F0BFE02000006C
:103F70006D4BF7B59D446D4B00206B44D860586A7B
:103F8000170080689860196A69480818D861407CF1
:103F9000012806D06748654B2C339D44F0BC08BC13
:103FA0001847624B6B44186A80309861FCF714FB29
:103FB0005E4BC5226B441B6A92019D18EA6A01267A
:103FC0003100824200D80021584B21206B441A6AEC
:103FD00000021418A1719869FCF706FB012109037E
:103FE000884201DA012000E00020504B6B44186148
:103FF000E179012000290CD1E178002909D061780C
:10400000002906D1A179002903D1617A002900D1C4
:104010000020464B83216B441A6A890152180028FC
:104020005A6104D0203303CBFCF7E6FA29E0E86BB1
:10403000431C05D03D4B6B445A69916B814221D2A0
:104040003A4BE96A6B449A6902A8FCF7DDFA374BF0
:10405000E86A6B445A69916B09189163196A8A6816
:1040600000922E6B0F6E02009968330002A8FFF7D2
:1040700089FC002816D02D4B6B44586A196AFCF74E
:10408000CBFA0700002F16D1284B6B44D869007C6F
:1040900000280AD001280ED1186900280BD0012071
:1040A000D86008E02348401D04E0204B6B44186AA8
:1040B000FCF7BAFA0700E86B431C08D01B4B012140
:1040C0006B445A69926B824211D200210FE0174B68
:1040D0006B449869FCF780FA22780021002A02D10B
:1040E0006279002A03D0EA6A824200D90121617212
:1040F000607A00280CD0104C2078002808D10B4B97
:104100006B44186AFCF720FA07000126267008E0C5
:10411000064B6B44D868002803D0186AFCF70CFAE9
:104120000700380037E70000E0F7FFFF0008000055
:10413000E020000001810000E079F0BFF7B5040045
:1041400088682121008809026718002600250028B8
:1041500002D01B48029000E0BE701A480299201855
:10416000C180FFF725FC002800D101257878164F83
:10417000002803D00120207378700BE0002D04D1BB
:104180002000FCF709FA0290F4E72000FCF704FA9B
:10419000029026730D48201886832000FCF7ECF966
:1041A0000A49200084398030FCF7EEF98320800131
:1041B0002018466386630298FEBC08BC18470000BE
:1041C0000E41000060310000E079F0BFE020000007
:1041D00070B506000C000025FCF7EEFA0023E15E46
:1041E0000423E05E762813D008DC0E2810D01228B5
:1041F0000ED013280CD016280DD109E0782807D04E
:104200009A2803D09C2801D09E2804D1294C36E05E
:10421000284C641E33E03100FCF746F901042548C0
:104220000914FF221332401C9142A1803ED0CB1FC3
:10423000FF3BFFF7AFFB09060B0C0B120B180B1E15
:104240000B002A0021003000FCF736F916E02A00A6
:1042500021003000FCF74CFA10E02A002100300069
:10426000FCF74EFA0AE02A0021003000FCF73CF986
:1042700004E02100104A300000F024F80400FFF7A9
:1042800097FB002811D10D48417801290DD1002557
:104290004570C52080013018C561856145613000D9
:1042A00007498030FCF770F93573200070BC08BCFA
:1042B000184700000281000002410000E079F0BFD1
:1042C0005C20000070B50E0005008C68100022D143
:1042D000212109026918CA79002A228814D0002AEB
:1042E00001D0114817E00022CA7110496918497CB1
:1042F000002905D001290ED12800FCF765F90AE054
:104300002800FCF759F906E0002A02D00122CA7100
:1043100001E00548401C020031002388280000F01D
:1043200007F870BC08BC184706410000E0200000F8
:1043300070B5060088680C0002804380FF203100C1
:1043400015001030FCF730FA010408480914301841
:104350001E23C05EA2680423FCF732FA002800D0B6
:10436000034D280070BC08BC18470000E020000086
:1043700007810000F8B50700886816000D000024CA
:104380000280022B438002D99B1E1C04240C39009E
:10439000FF200A30FCF708FA010408481E233818E9
:1043A000C05E0914AA68A31DFCF70AFA002800D011
:1043B000034E3000F8BC08BC18470000E0200000A5
:1043C00007810000FFB581B00AAEC0CE00252349A9
:1043D000040005734573012061180874487420486F
:1043E00083222018058045808580C580C5208001F6
:1043F00020188562C562056392014563A218856332
:1044000055639563C56185614561212000022018CF
:10441000857202208D83C883104920008439803042
:10442000FCF7B2F82000FCF7A7F830222000029930
:104430005030FCF731F93022200003992030FCF78E
:104440002BF90498211D41C106482770057045705D
:1044500005B0F0BC08BC002018470000E0200000B8
:1044600060310000E079F0BF5C009FE50020E0E3F0
:10447000082080E554109FE5043091E5083083E37F
:10448000043081E50030A0E3083080E5082080E5B5
:1044900004C091E508C08CE304C081E5083080E5E4
:1044A000082080E504C091E510C0CCE304C081E59C
:1044B000083080E5082080E5042091E5022B82E3A6
:1044C000042081E5083080E51EFF2FE1000300F89D
:1044D000000600F82C209FE524109FE50030E0E363
:1044E000000050E300C0A0E3083082E5000091E541
:1044F000020BC003020B8013000081E508C082E5B7
:104500001EFF2FE1000600F8000300F8F0472DE938
:10451000B8D04DE20C508DE201A0A0E10070A0E304
:104520000040A0E1CFF0FFEBDC609FE50000A0E3DE
:10453000010080E2060050E1FCFFFFBA000000EF3E
:10454000C9F0FFEB060050E30000001AFEFFFFEA8F
:104550008C008DE2C5F0FFEB0680A0E30090A0E3A5
:10456000150000EAB480CDE104108DE28C008DE2EC
:10457000B690CDE1B840CDE1BDF0FFEB8020A0E3E7
:104580000C108DE28C008DE2BAF0FFEB000050E3DE
:104590000600000A0000A0E3010080E2060050E1EE
:1045A000FCFFFFBA8C008DE2B0F0FFEB020000EAE6
:1045B000B200D5E1010050E30300000A000057E318
:1045C0000100001A000054E3E5FFFF1A0400A0E315
:1045D000B000CDE10200A0E3B200CDE18C008DE29D
:1045E0000D10A0E1A2F0FFEB8C008DE2A2F0FFEB3A
:1045F000000054E30400D5150A00A0019FF0FFEB72
:10460000B8D08DE2F047BDE81EFF2FE120A10700E2
:1046100070402DE90040A0E1000090E50050A0E3CB
:10462000341090E5020A11E30250A0030D00000AC5
:10463000021CA0E33C1080E5001094E5020AA0E310
:104640003C0081E5100094E571F1FFEB100094E56A
:104650006FF1FFEB180094E51C1094E5B000D0E179
:10466000000051E10150A0330500A0E17040BDE819
:104670001EFF2FE100009FE51EFF2FE13834F0BF41
:1046800000009FE51EFF2FE11833F0BF00009FE5FB
:104690001EFF2FE15434F0BF00009FE51EFF2FE105
:1046A0006434F0BF70402DE910608DE240C09FE59A
:1046B000700096E800E09CE500E0C0E504009CE5A1
:1046C0000000C1E508009CE50000C2E50400A0E38D
:1046D0000000C3E50200A0E30000C4E514009FE56C
:1046E000000085E52500A0E3000086E57040BDE8F8
:1046F0001EFF2FE19834F0BF512500003C402DE90A
:104700000050A0E10040A0E3840084E0800085E048
:104710000010A0E35DF1FFEB014084E20C0054E3E4
:10472000F8FFFFBA0000A0E35300C5E5B005C5E1FE
:104730004800C5E5C830A0E30020A0E35200C5E56D
:104740000C008DE80A30A0E30500A0E10210A0E310
:104750004FF1FFEB3C40BDE81EFF2FE1342090E518
:10476000303090E5241080E2030052E103C042E0C3
:10477000003091350030A02303309CE01000A003EE
:104780001EFF2F01083091E504C091E5000052E3BF
:104790000010910501104212011041020120A0E316
:1047A0009C3121E0082081E50E21C0E50000A0E356
:1047B0001EFF2FE170402DE9100080E3025BC0E393
:1047C0001850C5E3050001E0D8109FE5D8C09FE56B
:1047D0001000D0E300E0E0E30040A0E31C00000A8A
:1047E000000052E308E08CE5382091E52E6A00E0F5
:1047F0000620C20106208211382081E508408CE5A0
:10480000000053E308E08CE53C2091E5003AA0E18C
:10481000233AA0E10320C201032082113C2081E55C
:1048200008408CE508E08CE5302091E5000AA0E125
:10483000200AA0E1002082E1302081E508408CE5DB
:1048400008E08CE5342091E50000C2E1340081E508
:1048500008408CE508E08CE5040091E5052AA0E11C
:10486000222AA0E10200C0E1040081E508408CE5B5
:1048700008E08CE5100091E5100081E508408CE52A
:1048800008E08CE51C0091E51C0081E508408CE502
:1048900008E08CE5280091E5280081E508408CE5DA
:1048A0007040BDE81EFF2FE1000600F8000300F88D
:1048B0001000C0E302CB80E35C009FE50020E0E352
:1048C00008C08CE3082080E550109FE5043091E596
:1048D000023603E022CA0CE003308CE1043081E5AB
:1048E0000030A0E3083080E5082080E510C091E5A5
:1048F00010C081E5083080E5082080E51CC091E506
:104900001CC081E5083080E5082080E5282091E57D
:10491000282081E5083080E51EFF2FE1000300F824
:10492000000600F802CBC0E35C009FE50020E0E356
:1049300018C0CCE3082080E550109FE5003091E5D9
:10494000023603E022CA0CE003308CE1003081E53E
:104950000030A0E3083080E5082080E50CC091E538
:104960000CC081E5083080E5082080E518C091E59D
:1049700018C081E5083080E5082080E5242091E515
:10498000242081E5083080E51EFF2FE1000300F8B8
:10499000000600F844209FE50010A0E30000A0E31B
:1049A0000130A0E300C192E700005CE31310811125
:1049B000010080E2110050E3F9FFFF3A20009FE57B
:1049C0000020A0E3001080E5C02080E5082080E5FD
:1049D000C42080E50C009FE5060080E81EFF2FE163
:1049E0004457F0BF000300F8B034F0BFF0412DE9A8
:1049F0000040A0E1D000D0E10270A0E10160A0E1A0
:104A0000010050E3010070130050E0E31100000AC0
:104A1000020C84E2520080E21420A0E30610A0E120
:104A2000DDFBFFEB250EA0E3B47080E10600A0E102
:104A300001F1FFEB010050E30600001A4E02C4E54D
:104A40001C109FE50400A0E1FCF0FFEBD000D4E1D6
:104A5000F041BDE81EFF2FE10000E0E30050C4E597
:104A6000FAFFFFEAEC34F0BF10402DE90040A0E16E
:104A7000D000D0E10020E0E3000050E3010070131B
:104A80000A00000A4E02D4E5010050E30700001AB4
:104A9000000051E320109F0520109F150400A0E1A5
:104AA000E6F0FFEBD000D4E11040BDE81EFF2FE19F
:104AB0000000E0E30020C4E5FAFFFFEA9C35F0BF08
:104AC0006C35F0BF10402DE90040A0E1D000D0E1EE
:104AD0000010E0E3000050E3010070130800000A3A
:104AE0004E02D4E5010050E30500001A1C109FE5BA
:104AF0000400A0E1D1F0FFEBD000D4E11040BDE80C
:104B00001EFF2FE10000E0E30010C4E5FAFFFFEA1A
:104B10003C35F0BFF84F2DE9DC419FE50000A0E3F4
:104B20000170A0E34C0084E59EF0FFEB000050E331
:104B30005800000AC4519FE50300A0E301BAA0E3B6
:104B40000000C4E53CB085E5300095E5010A80E34E
:104B5000300085E50500A0E320EEFFEBA0119FE506
:104B6000006281E00C0096E50300C0E30C0086E5DE
:104B7000200094E541104BE2019000E0D9F0FFEBFA
:104B8000241084E20900A0E1CBF0FFEB74719FE5F3
:104B900001A000E2080087E20080E0E368219FE5D1
:104BA000981000E1021081E1081087E5C40087E257
:104BB000981000E1FF1081E3C41087E5101094E520
:104BC000240084E2C8F0FFEB0AA000E0C7F0FFEB8E
:104BD000101094E5240084E2C5F0FFEB0AA000E089
:104BE000C40087E2981000E1FF10C1E3C41087E51C
:104BF000080087E214219FE5981000E1021001E00F
:104C0000081087E5BBF0FFEB241084E20900A0E167
:104C1000B0F0FFEB0A7000E03CB085E5300095E5B0
:104C2000010AC0E3300085E5000095E5010080E35E
:104C3000000085E5000095E5020080E3000085E5C1
:104C4000000095E5040080E3000085E5000095E59F
:104C50000A00C0E3000085E5000095E51400C0E30C
:104C6000000085E5000095E50100C0E3000085E552
:104C7000021AA0E33C1085E50C0096E5010080E3F4
:104C80000C0086E50100A0E34C0084E5240095E5D6
:104C90003C1085E5130000EA97F0FFEB000050E3BD
:104CA0000D00000A0200A0E30000C4E50400D4E502
:104CB0000020A0E3241084E289F0FFEB015000E221
:104CC0008AF0FFEB0300D4E50020A0E3241084E287
:104CD00083F0FFEB057000E0020000EA0100A0E3B2
:104CE0000000C4E581F0FFEB0000A0E30000C4E594
:104CF0000700A0E1F84FBDE81EFF2FE1D436F0BF5A
:104D0000000D00F8000200F8000300F8FDFF0100AC
:104D10000200FEFF04E02DE5C4EDFFEB1D10A0E353
:104D2000910000E014109FE5001091E5000181E082
:104D3000010C80E2F404D0E104E09DE41EFF2FE1C9
:104D4000F035F0BF14309FE5003080E510009FE59E
:104D5000000081E50C009FE5000082E51EFF2FE1C9
:104D6000DC78F0BFD09A01C0E09A01C0FEB5040023
:104D700040690E00002500280DD0A069002802D14E
:104D8000B068A0616FE0E069002802D1B068E0611E
:104D900069E0374D67E0312080012718787B0028D3
:104DA000019004D12900300000F05AFA2EE0B168D9
:104DB0002000FCF741FA050055D121003000FCF736
:104DC00043FA0500787B019988424CD02949611843
:104DD0000291A3214901671827496618002817D0B6
:104DE00001283ED1B87D002834D001283BD1B07ACB
:104DF000002838D1212080012018426801218B022F
:104E0000D218917241682000FCF726FA05002AE0CA
:104E1000B87D002802D0B07A002824D01748211885
:104E20002000FCF721FA05000120F0720220A0709A
:104E3000B87D002808D10198022805D10023E05E42
:104E4000029A2921FBF7BCFCB07A00280BD0002085
:104E5000707208E00023E05E029A2921FBF7B0FCA3
:104E600001E0034D0B3D2800FEBC08BC18470000C4
:104E700031800000701E0100401601005014000037
:104E8000F3B581B0029904008E683349002065189B
:104E9000A3212A8849016718A988002A1DD1002961
:104EA0001DD1616900291CD1B97D00291ED130783E
:104EB00000280CD02000FCF72FFA2000FCF734FA71
:104EC000002811D12000FCF737FA00280CD101226C
:104ED000711C2000FCF738FA04E0002901D008001A
:104EE00000E01000002801D00121A170697A00299A
:104EF00000D01A486169002901D018480930020021
:104F000002982100FCF728FA060012D1B87D00288B
:104F100013D001280DD121208001201841680127DC
:104F2000BA0289188F7241682000FCF795F90600D3
:104F30006F723000FEBC08BC184731208001201879
:104F4000407B0128F5D1064900236218E05E292143
:104F5000FBF736FCEDE70000401601004A40000078
:104F6000701E010038B52C48FEF71AFD040003D16D
:104F7000012038BC08BC1847284900206118A070DF
:104F8000088048808880A322C88052010872A21835
:104F90000123C872137350739073D073C8231082A7
:104FA000538290822922D201A218D0621B4A4872F1
:104FB0002032A2181070508088722000FCF744FA4A
:104FC000154902203839208004206118886213486E
:104FD000C83820180500FCF73FFA00208B22520247
:104FE000810009198918401C0A288D61F8D3200016
:104FF000FBF7A8FD09480021283822183430009218
:10500000C82220180123FCF72BFA0448243020186A
:10501000FCF7E2F90020ACE7781E01004016010021
:10502000F8B50423CF5E0500080000244C2F12D0F1
:1050300016DC252F29D008DC3B496E180E2F33D003
:10504000122F28D0132F6BD068E0272F03D02A2FE0
:1050500001D02C2F62D1210000F002F904005FE0A2
:105060009A2F4FD00BDC31495F2F51D0612F52D096
:10507000642F53D10A002900FCF706F9EEE79C2FB4
:1050800043D09E2F4AD12A4C4AE0284A121F2900B9
:10509000FCF70AF9E2E780680088002801D0234C79
:1050A000E41F0420348015E080680088002801D0C7
:1050B0001E4CA41FA320400128187480807D002866
:1050C0000AD001282CD11B4829182800FCF7E0F948
:1050D00004000320A87023E0317A01200027002972
:1050E00003D03772F072AF7003E0A870F07A002836
:1050F00016D0114900236A18E85E6321FBF760FBB4
:10510000F7720DE00A4C641E0AE0094CA41C07E08B
:10511000FCF7EAF8A2E7FCF7EFF89FE7044C0E3C37
:105120002000F8BC08BC1847401601004D400000A4
:105130002E80000054140000741E0100F8B50423F2
:10514000CF5E0500080000244C2F10D014DC252F62
:1051500029D006DC0E2F2FD0122F2AD0132F70D07B
:105160006DE0272F03D02A2F01D02C2F67D12100EB
:1051700000F076F8040064E034496E189A2F1ED0CF
:105180000BDC33495F2F54D0612F55D0642F56D19B
:105190000A002900FCF778F8ECE79C2F2BD09E2F13
:1051A0004DD12C4C4DE02A4A121F2900FCF77CF807
:1051B000E0E7284C0B3C44E0264CE41E41E08068CC
:1051C00022490090008820316F18002806D0204C1A
:1051D0000420A41E0021A87079800AE01E48291826
:1051E0002800FCF719F904000220A87000984088F4
:1051F0007880B48025E080680088002801D0144CB5
:10520000641E317A0120002905D000213172B1726B
:10521000F072A97003E0A870F07A0028E9D00F4975
:1052200000236A18E85E6321FBF7CAFA0021F172D5
:10523000DFE7FCF759F89DE7FCF75EF89AE7054CC5
:105240000E3C2000F8BC08BC1847000040160100C6
:105250004D4000002E80000050140000741E01001C
:1052600070B5040080680D00002808D0FBF7A4FA90
:105270000423E15E083444CC3300FBF7A1FA280094
:1052800070BC08BC18470000A3225201821810B459
:10529000137BD27B022B0BD1002A05D0032A05D029
:1052A000062A0CD111490AE0114908E0114906E02B
:1052B000002A08D0032A08D0062A00D10E4900226D
:1052C0008B24640203E00D49F9E70D49F7E79300E9
:1052D0001B181B1999619E31521C092AF7D30949E1
:1052E00041180019C16310BC70470000165DF0BF83
:1052F0004E73F0BF3268F0BF8857F0BFC06DF0BF8B
:10530000A462F0BF78150100FFB50E00140000255F
:1053100083B01F4F02952DE001784900795A890723
:1053200008D56946FCF718F9002803D06846FCF751
:105330001BF90290316808784200BA5AD20513D599
:10534000144B002102E0491C092903DA8A009A5C07
:105350008242F8D18800C2183100029B2000FCF77D
:105360000BF92D18241805E0481C306008782070CF
:10537000641C6D1C300003C8884202D803998D421A
:10538000CADB00202070280007B0F0BC08BC18471A
:10539000706F01C0146D01C0030052E33D00009A1C
:1053A00003C010E20800000A0130D1E402005CE30F
:1053B0000C2082E001C0D1940130C0E40130D1342E
:1053C000042042E201C0C0940130C034033011E235
:1053D0001D00000A042052E22E00003A03C031E70B
:1053E000020053E30800000A0F00008A2C34A0E1F9
:1053F00004C0B1E5042052E20C3C83E1043080E4B7
:10540000F9FFFF2A011081E2220000EA2C38A0E116
:1054100004C0B1E5042052E20C3883E1043080E49A
:10542000F9FFFF2A021081E21A0000EA2C3CA0E1F9
:1054300004C0B1E5042052E20C3483E1043080E47E
:10544000F9FFFF2A031081E2120000EA10402DE963
:10545000202052E20500003A1850B1281850A02828
:105460001850B1281850A02820205222F9FFFF2AF6
:1054700002CEB0E11850B1281850A0281800B14849
:105480001800A0481040BDE802CFB0E104309124DC
:10549000043080241EFF2F01822FB0E10120D1446F
:1054A0000130D12401C0D1240120C0440130C024E6
:1054B00001C0C0241EFF2FE10020A0E3040051E33F
:1054C0000800003A03C010E20C00000A04C06CE2BD
:1054D00002005CE30120C0E40120C0A40120C0C49C
:1054E0000C1041E0050000EA81CFB0E10120C024AA
:1054F0000120C0240120C0441EFF2FE10020A0E3B2
:1055000000402DE90230A0E102C0A0E102E0A0E1EC
:10551000201051E20C50A0280C50A028201051223D
:10552000FBFFFF2A011EB0E10C50A0280C00A04890
:105530000040BDE80111B0E1042080241EFF2F01CE
:105540000120C0440120C044400411E30120C014E4
:105550001EFF2FE1030010E3030011031700001AE0
:1055600000402DE950E29FE5042090E4043091E4EE
:105570000EC042E002C0CCE18EC31CE00300520129
:10558000F8FFFF0A0040BDE8030CA0E1020C50E068
:10559000FF0E1C030700001A0308A0E1020850E0F8
:1055A000FF0C1C030300001A0304A0E1020450E0F6
:1055B000FF081C03020053006000A0111EFF2FE132
:1055C0000120D0E40130D1E4010052E30300522174
:1055D0000400001A0120D0E40130D1E4010052E3BC
:1055E00003005221F5FFFF0A030042E01EFF2FE1F6
:1055F000013080E1030013E304E02DE50020A0E189
:105600000B00001AB0C19FE5043091E40CE043E0C8
:1056100003E0CEE18C031EE104308204F9FFFF0AAF
:10562000FF1013E20110C2E42334A011FBFFFF1AA4
:10563000070000EA0130D1E40130C2E4000053E386
:105640000300000A0130D1E40130C2E4000053E35A
:10565000F7FFFF1A0040BDE81EFF2FE101C080E206
:10566000030010E30500000A0110D0E4000051E33C
:105670000C0040001EFF2F01030010E3F9FFFF1A8A
:1056800034219FE5041090E4023041E00130C3E191
:10569000820313E1FAFFFF0A0C0040E0FF0011E370
:1056A000030040021EFF2F01FF0C11E30200400225
:1056B0001EFF2F01FF0811E3010040021EFF2FE132
:1056C000013080E1030013E304E02DE50D00001A32
:1056D000E4C09FE5020000EA040080E2041081E2D9
:1056E000042042E2040052E30030902500E09125BE
:1056F0000E0053210300001A0CE043E00330CEE11A
:105700008C0313E1F3FFFF0A000052E30000A00343
:105710000700000A0130D0E401C0D1E4010053E3E6
:105720000C0053210100001A012052E2F8FFFF1A79
:105730000C0043E00040BDE81EFF2FE1040052E3EF
:1057400001308021030013230900001A043090E483
:1057500004C091E40C0053E10200001A042042E26C
:10576000040052E3F8FFFF2A0C0053E1040040124A
:1057700004104112000052E30000A0031EFF2F019D
:10578000010012E3012082120300001A0130D0E46C
:1057900001C0D1E40C0053E10500001A0130D0E44F
:1057A00001C0D1E40C0053E10100001A022052E2D2
:1057B000F5FFFF1A0C0043E01EFF2FE1010101017C
:1057C000BC02F0BFB802F0BF000000000000000003
:1057D00000000000000000000000000000000000C9
:1057E000B402F0BFB002F0BFB002F0BF0000000092
:1057F00000000000000000000000000000000000A9
:10580000000000000100000064006400640000006B
:105810001900040000006400AC0DFA003C0FE8031E
:10582000AC0D94113C00410041005700480042007B
:105830003D003C004F004900120000005A000A00E1
:105840001C00900114058C0AF40114004600F92A8A
:10585000E9030100000000000000920246006E0013
:10586000A000B400C800FA00400104010E01C012FB
:1058700058021E005000C800200364000000010010
:105880000A0005009C04580226009CFF6AFF0100E4
:10589000C80064009600FA003C006400900100001B
:1058A000681001000000640057005000000046002E
:1058B000140000006B00AC0D1801740E9001800CF8
:1058C000101341003A004100570044003C003C00E6
:1058D0003D0055000A00050000005F000A001600A8
:1058E000F401E803FC08E80300005A0033268A02AA
:1058F0000100020000000000B6013C006E006E00D6
:10590000E6005401FA004001040104017E13B004D2
:1059100032005000900120036400000000000200EB
:1059200005009C041C021E00000000000000C800CE
:1059300064003C003C003C003C00900100009411DD
:10594000000000006400B4006400000014000A00BD
:1059500000006400CC10A0005C12580268102413F0
:1059600049004100460077006700440029004600D6
:105970006A001E000F0032005500000023007C0169
:105980004C04C409580214005000AC71D449010001
:10599000010000000000B6015000620091002C01DF
:1059A0005802FA004001040172015C12580214000E
:1059B0001E00A00020036400000003001700050083
:1059C00046055E012300B400B4000700C2019CFF3D
:1059D000DC00C2016400CC005E01280094110000CC
:1059E0003C006400DC00640000003C000500000096
:1059F000640062110401561358026211241340001E
:105A00003B0040005700490042002D003A0053007F
:105A10003C00120032001E00010020005E01E8037D
:105A2000DC05BC020000410010724C0401000600BD
:105A300000000000B601780082008C00E6005401EE
:105A4000FA00DC00FA00C800C012B00414005000D4
:105A5000640084036E0000000100080005000005DA
:105A60008A021E00000000000000FA009CFF3C00BB
:105A70003C003C006400900100002A12010041003B
:105A800064006E0064001E0014000A000000640040
:105A9000AC0DF000D80EB400041024134100340003
:105AA0004100570049003E0041003E004D006400A7
:105AB0000900460032000A0016009001E803B00415
:105AC000BC02000032005C2BF40101000400000065
:105AD0000000B60146005A008200B400C800FA0077
:105AE000400104010E01C01258020A005000640077
:105AF00020036400000001000A0005009C041C0251
:105B00001E00000000000000900164003C003C000A
:105B10003C003C0090010000941100003200410064
:105B20001D017800000028000A00000060005C12DF
:105B3000F401701770176211C01241003C0041005F
:105B400057005700490039003D0040004B000A0053
:105B50004B003200140014002C01E8033408BC028E
:105B600000001E001C25400601000500000000008A
:105B7000B6015F008200A000B400C800FA00400136
:105B800004010E01C012B0040A005000640020039A
:105B90006400000000000A0005009C04B6031E001B
:105BA0000000000000002C012C013C003C003C00E7
:105BB0003C00900100005C1201001E0064006E00B9
:105BC0006400000014000A0000006400AC0D5E01D7
:105BD0009411F401480DC0124100370041005700F4
:105BE000480043003E003D004D0049001200000007
:105BF0002800120005009001E8033408BC020000F0
:105C000050003F302F090100030000000000B601E2
:105C1000640078009600B4005E01FA0040010401BF
:105C20000E01C01258020A005000640052036400C2
:105C300000000100010005009C041C021E00000081
:105C40000000080064000A003C003C003C006400C6
:105C5000900100009411000046006400BE00640042
:105C60000A002800000000006400EC0FF00070172C
:105C70007017C80F70174B003C00410043005700DD
:105C80004600320039004D001E000A003C002D0085
:105C900005003200C201E803080790010000490036
:105CA000CE314C040100070000000000B6018C005A
:105CB000DC00F000E6005401FA0040010401040198
:105CC0007E1358021400500064008A02780000001D
:105CD0000100050005009C048A022D000000C2019D
:105CE000000012024B00C800C2012C013C00BC02A3
:105CF00000005014000014003200C30064000A00C9
:105D000014000A0000006400F8112C0170177017CD
:105D10006810C0123D003D00410057005700490087
:105D20003B003C00440064000A00500014001200D4
:105D30001600C201E803C40984033C003C00B42DF2
:105D40004C040100080000000000B6017800820049
:105D50008C00E6005401FA00DC00FA00C800C01212
:105D6000B00414005000640084036E0000000200C0
:105D70000200050046055E011E0000000000000054
:105D8000900164003C003C003C003C00900100009D
:105D9000F2120100000064006400640000001900B9
:105DA000040000006400AC0DFA003C0FE803AC0DE9
:105DB00094113C0041004100570057003F0039005A
:105DC000390053004900120000005A000A001C006C
:105DD000900114058C0AF40114004600F92AE90325
:105DE0000100000000000000920246006E00A000CA
:105DF000B400C800FA00400104010E01C0125802AC
:105E00001E005000C80020036400000001000A00CA
:105E100005009C04580226009CFF6AFF0100C80090
:105E200064009600FA003C006400900100006810D5
:105E300001000000640057005000000046001400FC
:105E400000006B00AC0D1801740E9001800C101353
:105E500041003A00410057003F00380037003E0043
:105E600057000A00050000005F000A001600F40158
:105E7000E803FC08E80300005A0033268A02010008
:105E8000020000000000B6013C006E006E00E6005B
:105E90005401FA004001040104017E13B0043200F1
:105EA0005000900120036400000000000200050083
:105EB0009C041C021E00000000000000C8006400DA
:105EC0003C003C003C003C009001000094110000AC
:105ED00000006400B4006400000014000A00000028
:105EE0006400CC10A0005C12580268102413470014
:105EF0003F00440077007600590027003F00610012
:105F00001E000F0032005500000023007C014C04ED
:105F1000C409580214005000AC71D44901000100BA
:105F200000000000B6015000620091002C015802F0
:105F3000FA004001040172015C12580214001E00B4
:105F4000A0002003640000000300170005004605C0
:105F50005E012300B400B4000700C2019CFFDC0016
:105F6000C2016400CC005E012800941100003C00D6
:105F70006400DC00640000003C00050000006400D8
:105F80006211040156135802621124133F003A00B3
:105F90003F005700570057002A0031004F003C00D7
:105FA000120032001E00010020005E01E803DC0543
:105FB000BC020000410010724C0401000600000009
:105FC0000000B601780082008C00E6005401FA005F
:105FD000DC00FA00C800C012B004140050006400D5
:105FE00084036E00000001000800050000058A021D
:105FF0001E00000000000000FA009CFF3C003C0076
:106000003C006400900100002A120100410064007D
:106010006E0064001E0014000A0000006400AC0D55
:10602000F000D80EB40004102413410034004100E5
:1060300057003F0033003E003D0057006400090058
:10604000460032000A0016009001E803B004BC02CA
:10605000000032005C2BF40101000400000000008D
:10606000B60146005A008200B400C800FA004001A0
:1060700004010E01C01258020A00500064002003FF
:106080006400000001000A0005009C041C021E00C0
:10609000000000000000900164003C003C003C0057
:1060A0003C009001000094110000320041001D01ED
:1060B0007800000028000A00000060005C12F40173
:1060C000701770176211C01240003B00400055006D
:1060D000570057003600380042004B000A004B00C2
:1060E0003200140014002C01E8033408BC02000044
:1060F0001E001C2540060100050000000000B6013E
:106100005F008200A000B400C800FA004001040152
:106110000E01C012B0040A005000640020036400A5
:10612000000000000A0005009C04B6031E000000E9
:10613000000000002C012C013C003C003C003C0015
:10614000900100005C1201001E0064006E006400FB
:10615000000014000A0000006400AC0D5E01941100
:10616000F401480DC01241003700410057005700AC
:1061700040003A003A005100490012000000280097
:10618000120005009001E8033408BC020000500032
:106190003F302F090100030000000000B601640039
:1061A00078009600B4005E01FA00400104010E017F
:1061B000C01258020A00500064005203640000003C
:1061C0000100010005009C041C021E0000000000EC
:1061D000080064000A003C003C003C0064009001A0
:1061E00000009411000046006400BE0064000A0034
:1061F0002800000000006400EC0FF000701770171A
:10620000C80F70174B003C00410043005700570077
:106210002E0035004B001E000A003C002D0005003A
:106220003200C201E8030807900100004900CE31A6
:106230004C040100070000000000B6018C00DC00E7
:10624000F000E6005401FA004001040104017E134D
:1062500058021400500064008A0278000000010017
:10626000050005009C048A022D000000C201000008
:1062700012024B00C800C2012C013C00BC0200000D
:106280005014000014003200C30064000A0014001F
:106290000A0000006400F8112C01701770176810D4
:1062A000C0123D003D004100570057005700370025
:1062B0003700450064000A00500014001200160068
:1062C000C201E803C40984033C003C00B42D4C0423
:1062D0000100080000000000B601780082008C0078
:1062E000E6005401FA00DC00FA00C800C012B00455
:1062F00014005000640084036E00000002000200DD
:10630000050046055E011E0000000000000090012F
:1063100064003C003C003C003C0090010000F21294
:106320000100000064006400640000001900040023
:1063300000006400AC0DFA003C0FE803AC0D9411B2
:106340003C00410041005700480042003D003C0035
:106350004F004900120000005A000A001C00900182
:1063600014058C0AF40114004600F92AE90301001F
:10637000000000000000920246006E00A000B40081
:10638000C800FA00400104010E01C01258021E00AC
:106390005000C80020036400000001000A0005004E
:1063A0009C04580226009CFF6AFF0100C80064009C
:1063B0009600FA003C0064009001000068100100A3
:1063C0000000640057005000000046001400000068
:1063D0006B00AC0D1801740E9001800C101341007D
:1063E0003A004100570044003B003C003F0054008D
:1063F0000A00050000005F000A001600F401E8032F
:10640000FC08E80300005A0033268A02010002005B
:1064100000000000B6013C006E006E00E600540172
:10642000FA004001040104017E13B0043200500060
:1064300090012003640000000000020005009C049D
:106440001C021E00000000000000C80064003C00A8
:106450003C003C003C009001000094110000000052
:106460006400B4006400000014000A00000064002E
:10647000CC10A0005C12580268102413490041009F
:106480004600770067004300290047006A001E00AD
:106490000F0032005500000023007C014C04C409A9
:1064A000580214005000AC71D449010001000000F2
:1064B0000000B6015000620091002C015802FA0061
:1064C0004001040172015C12580214001E00A00079
:1064D00020036400000003001700050046055E016C
:1064E0002300B400B4000700C2019CFFDC00C2011D
:1064F0006400CC005E012800941100003C006400A0
:10650000DC00640000003C00050000006400621133
:106510000401561358026211241341003C0041004B
:106520005700490042002D00390052003C00120083
:1065300032001E00010020005E01E803DC05BC0201
:106540000000410010724C04010006000000000031
:10655000B601780082008C00E6005401FA00DC00ED
:10656000FA00C800C012B004140050006400840394
:106570006E00000001000800050000058A021E00F0
:10658000000000000000FA009CFF3C003C003C00C2
:106590006400900100002A120100410064006E00B6
:1065A00064001E0014000A0000006400AC0DF0003E
:1065B000D80EB400041024134100340041005700E9
:1065C00049003F0040003E004C00640009004600C6
:1065D00032000A0016009001E803B004BC0200007B
:1065E00032005C2BF4010100040000000000B60141
:1065F00046005A008200B400C800FA0040010401BD
:106600000E01C01258020A0050006400200364000A
:10661000000001000A0005009C041C021E0000008E
:1066200000000000900164003C003C003C003C0085
:106630009001000094110000320041001D0178001B
:10664000000028000A00000060005C12F4017017CE
:1066500070176211C01241003C0041005700570002
:1066600048003A003C0041004B000A004B00320059
:10667000140014002C01E8033408BC0200001E00C2
:106680001C2540060100050000000000B6015F0067
:106690008200A000B400C800FA00400104010E010D
:1066A000C012B0040A00500064002003640000001F
:1066B00000000A0005009C04B6031E000000000054
:1066C00000002C012C013C003C003C003C009001EF
:1066D00000005C1201001E0064006E0064000000F7
:1066E00014000A0000006400AC0D5E019411F40176
:1066F000480DC012410037004100570048004300D8
:106700003E003C004E00490012000000280012002C
:1067100005009001E8033408BC02000050003F303F
:106720002F090100030000000000B601640078009A
:106730009600B4005E01FA00400104010E01C0128F
:1067400058020A0050006400520364000000010077
:10675000010005009C041C021E000000000008004F
:1067600064000A003C003C003C0064009001000012
:106770009411000046006400BE0064000A00280076
:10678000000000006400EC0FF00070177017C80FD5
:1067900070174B003C004100430057004700320097
:1067A00039004B001E000A003C002D00050032009D
:1067B000C201E8030807900100004900CE314C04F3
:1067C0000100070000000000B6018C00DC00F000B2
:1067D000E6005401FA004001040104017E1358024E
:1067E0001400500064008A027800000001000500D7
:1067F00005009C048A022D000000C2010000120264
:106800004B00C800C2012C013C00BC020000501427
:10681000000014003200C30064000A0014000A00E3
:1068200000006400F8112C01701770176810C01276
:106830003D003D0041005700570048003C003B0030
:10684000440064000A005000140012001600C20147
:10685000E803C40984033C003C00B42D4C0401004F
:10686000080000000000B601780082008C00E600FD
:106870005401FA00DC00FA00C800C012B004140091
:106880005000640084036E00000002000200050056
:1068900046055E011E00000000000000900164003B
:1068A0003C003C003C003C0090010000F212010062
:1068B000000064006400640000001900040000008F
:1068C0006400AC0DFA003C0FE803AC0D94113C00E1
:1068D00041004100570057003F0039003A00510085
:1068E0004900120000005A000A001C009001140523
:1068F0008C0AF40114004600F92AE90301000000A3
:1069000000000000920246006E00A000B400C80023
:10691000FA00400104010E01C01258021E0050008E
:10692000C80020036400000001000A0005009C0468
:10693000580226009CFF6AFF0100C8006400960010
:10694000FA003C00640090010000681001000000A3
:1069500064005700500000004600140000006B0067
:10696000AC0D1801740E9001800C101341003A0018
:10697000410057003F00380037003D0057000A0033
:10698000050000005F000A001600F401E803FC089F
:10699000E80300005A0033268A02010002000000CA
:1069A0000000B6013C006E006E00E6005401FA00E3
:1069B0004001040104017E13B00432005000900134
:1069C0002003640000000000020005009C041C027B
:1069D0001E00000000000000C80064003C003C00F5
:1069E0003C003C0090010000941100000000640095
:1069F000B4006400000014000A0000006400CC1021
:106A0000A0005C1258026810241347003F004400A5
:106A100077007600590027003F0061001E000F003C
:106A200032005500000023007C014C04C4095802C8
:106A300014005000AC71D4490100010000000000B6
:106A4000B6015000620091002C015802FA0040018A
:106A5000040172015C12580214001E00A000200301
:106A60006400000003001700050046055E012300D6
:106A7000B400B4000700C2019CFFDC00C201640046
:106A8000CC005E012800941100003C006400DC0092
:106A9000640000003C000500000064006211040175
:106AA000561358026211241340003B0040004C0072
:106AB00057005700290030004F003C001200320000
:106AC0001E00010020005E01E803DC05BC0200009E
:106AD000410010724C040100060000000000B601E5
:106AE000780082008C00E6005401FA00DC00FA0015
:106AF000C800C012B00414005000640084036E008B
:106B0000000001000800050000058A021E000000C8
:106B100000000000FA009CFF3C003C003C006400C8
:106B2000900100002A120100410064006E00640020
:106B30001E0014000A0000006400AC0DF000D80E26
:106B4000B4000410241341003400410057003F00FA
:106B500033003E003D00570064000900460032004B
:106B60000A0016009001E803B004BC0200003200E5
:106B70005C2BF4010100040000000000B601460097
:106B80005A008200B400C800FA00400104010E015E
:106B9000C01258020A005000640020036400000084
:106BA00001000A0005009C041C021E0000000000F9
:106BB0000000900164003C003C003C003C0090015F
:106BC000000094110000320041001D017800000017
:106BD00028000A00000060005C12F40170177017B2
:106BE0006211C01240003B004000570057005700A0
:106BF0003600380042004B000A004B0032001400FF
:106C000014002C01E8033408BC0200001E001C25FF
:106C100040060100050000000000B6015F00820090
:106C2000A000B400C800FA00400104010E01C01227
:106C3000B0040A005000640020036400000000005B
:106C40000A0005009C04B6031E00000000000000BE
:106C50002C012C013C003C003C003C009001000059
:106C60005C1201001E0064006E006400000014004D
:106C70000A0000006400AC0D5E019411F401480D9F
:106C8000C0124100370041005700570040003A0051
:106C90003A005100490012000000280012000500CF
:106CA0009001E8033408BC02000050003F302F0977
:106CB0000100030000000000B601640078009600A7
:106CC000B4005E01FA00400104010E01C012580236
:106CD0000A0050006400520364000000010001003B
:106CE00005009C041C021E00000000000800640057
:106CF0000A003C003C003C0064009001000094113C
:106D0000000046006400BE0064000A002800000085
:106D100000006400EC0FF00070177017C80F7017B8
:106D20004B003C0041004300570057002E00350047
:106D30004A001E000A003C002D0005003200C2017E
:106D4000E8030807900100004900CE314C0401001F
:106D5000070000000000B6018C00DC00F000E60037
:106D60005401FA004001040104017E13580214008A
:106D7000500064008A027800000001000500050050
:106D80009C048A022D000000C201000012024B0088
:106D9000C800C2012C013C00BC02000050140000DD
:106DA00014003200C30064000A0014000A0000004E
:106DB0006400F8112C01701770176810C0123D00A4
:106DC0003D0041005700570057003800360044008E
:106DD00064000A005000140012001600C201E8030B
:106DE000C40984033C003C00B42D4C04010008009D
:106DF00000000000B601780082008C00E60054011B
:106E0000FA00DC00FA00C800C012B0041400500000
:106E1000640084036E0000000200020005004605C5
:106E20005E011E00000000000000900164003C00B4
:106E30003C003C003C0090010000F2120100000008
:106E40006400640064000000190004000000640095
:106E5000AC0DFA003C0FE803AC0D941139003E0074
:106E60003E005700450042003E003D0050004900F2
:106E7000120000005A000A001C00900114058C0A40
:106E8000F40114004600F92AE903010000000000A3
:106E90000000920246006E00A000B400C800FA0094
:106EA000400104010E01C01258021E005000C8002B
:106EB00020036400000001000A0005009C04580241
:106EC00026009CFF6AFF0100C80064009600FA00DB
:106ED0003C006400900100006810010000006400A4
:106EE0005700500000004600140000006B00AC0D7D
:106EF0001801740E9001800C101341003A004100FB
:106F00005700400042003F003F0053000A000500C8
:106F100000005F000A001600F401E803FC08E80323
:106F200000005A0033268A0201000200000000001F
:106F3000B6013C006E006E00E6005401FA0040010C
:106F4000040104017E13B0043200500090012003BC
:106F5000640000000000020005009C041C021E00EA
:106F6000000000000000C80064003C003C003C0041
:106F70003C00900100009411000000006400B40087
:106F80006400000014000A0000006400CC10A0009F
:106F90005C12580268102413410039003E0057006B
:106FA00046003D0046003E0052001E000F00320029
:106FB0005500000023007C014C04C4095802140051
:106FC0005000AC71D4490100010000000000B6017E
:106FD0005000620091002C015802FA0040010401A7
:106FE00072015C12580214001E00A000200364000D
:106FF000000003001700050046055E012300B400F1
:10700000B4000700C2019CFFDC00C2016400CC0098
:107010005E012800941100003C006400DC00640064
:1070200000003C00050000006400621104015613DA
:1070300058026211241341003C00410057004400F3
:10704000400042003F0051003C00120032001E0090
:10705000010020005E01E803DC05BC0200004100E5
:1070600010724C040100060000000000B601780018
:1070700082008C00E6005401FA00DC00FA00C8002F
:10708000C012B00414005000640084036E000000BD
:1070900001000800050000058A021E000000000033
:1070A0000000FA009CFF3C003C003C0064009001A2
:1070B00000002A120100410064006E0064001E00FE
:1070C00014000A0000006400AC0DF000D80EB400FB
:1070D00004102413410034004100570049004000CF
:1070E00042003D004B0064000900460032000A00E7
:1070F00016009001E803B004BC02000032005C2BD3
:10710000F4010100040000000000B60146005A002E
:107110008200B400C800FA00400104010E01C01250
:1071200058020A00500064002003640000000100BF
:107130000A0005009C041C021E0000000000000064
:10714000900164003C003C003C003C0090010000C9
:1071500094110000320041001D0178000000280059
:107160000A00000060005C12F401701770176211D1
:10717000C01241003C004100570057004600430048
:107180003C0040004B000A004B0032001400140089
:107190002C01E8033408BC0200001E001C25400638
:1071A0000100050000000000B6015F008200A000A1
:1071B000B400C800FA00400104010E01C012B0047E
:1071C0000A005000640020036400000000000A0070
:1071D00005009C04B6031E000000000000002C0106
:1071E0002C013C003C003C003C00900100005C1283
:1071F00001001E0064006E006400000014000A001C
:1072000000006400AC0D5E019411F401480DC01241
:1072100041003700410057004800420040003D0057
:107220004E004900120000002800120005009001E5
:10723000E8033408BC02000050003F302F09010071
:10724000030000000000B601640078009600B4005E
:107250005E01FA00400104010E01C01258020A004A
:1072600050006400520364000000010001000500AA
:107270009C041C021E0000000000080064000A00BC
:107280003C003C003C0064009001000094110000B0
:1072900046006400BE0064000A00280000000000F0
:1072A0006400EC0FF00070177017C80F70174100E2
:1072B000320037004300570044004D0039004D00B4
:1072C0001E000A003C002D0005003200C201E80348
:1072D0000807900100004900CE314C04010007006E
:1072E00000000000B6018C00DC00F000E600540154
:1072F000FA004001040104017E13580214005000FA
:1073000064008A02780000000100050005009C046A
:107310008A022D000000C201000012024B00C800CA
:10732000C2012C013C00BC020000501400001400FB
:107330003200C30064000A0014000A000000640068
:10734000F8112C01701770176810C0123D003D0035
:10735000410057005700450044003B0045006400D1
:107360000A005000140012001600C201E803C4090C
:1073700084033C003C00B42D4C04010008000000D4
:107380000000B601780082008C00E6005401FA008B
:10739000DC00FA00C800C012B00414005000640001
:1073A00084036E00000002000200050046055E0135
:1073B0001E00000000000000900164003C003C0042
:1073C0003C003C0090010000F2120100000064004B
:1073D0006400640000001900040000006400AC0DAB
:1073E000FA003C0FE803AC0D94113C004100410051
:1073F000530057003B0037003E0053004900120085
:1074000000005A000A001C00900114058C0AF401C7
:1074100014004600F92AE903010000000000000002
:10742000920246006E00A000B400C800FA004001BD
:1074300004010E01C01258021E005000C8002003B3
:107440006400000001000A0005009C0458022600A8
:107450009CFF6AFF0100C80064009600FA003C002F
:1074600064009001000068100100000064005700F3
:10747000500000004600140000006B00AC0D180125
:10748000740E9001800C101341003A004100570027
:107490003E003D003900400057000A000500000092
:1074A0005F000A001600F401E803FC08E80300008E
:1074B0005A0033268A020100020000000000B601D3
:1074C0003C006E006E00E6005401FA004001040129
:1074D00004017E13B00432005000900120036400C8
:1074E00000000000020005009C041C021E000000B9
:1074F00000000000C80064003C003C003C003C0070
:10750000900100009411000000006400B4006400C9
:10751000000014000A0000006400CC10A0005C12FF
:10752000580268102413410039003E0057005700EC
:1075300057004200320048001E000F003200550084
:10754000000023007C014C04C409580214005000C0
:10755000AC71D4490100010000000000B6015000E8
:10756000620091002C015802FA00400104017201EE
:107570005C12580214001E00A000200364000000EA
:1075800003001700050046055E012300B400B400A7
:107590000700C2019CFFDC00C2016400CC005E0158
:1075A0002800941100003C006400DC00640000002E
:1075B0003C000500000064006211040156135802EB
:1075C0006211241341003C0041005700570057004E
:1075D0003C00360045003C00120032001E00010055
:1075E00020005E01E803DC05BC02000041001072CF
:1075F0004C040100060000000000B6017800820083
:107600008C00E6005401FA00DC00FA00C800C01249
:10761000B00414005000640084036E0000000100F8
:107620000800050000058A021E000000000000009E
:10763000FA009CFF3C003C003C006400900100000C
:107640002A120100410064006E0064001E00140054
:107650000A0000006400AC0DF000D80EB400041065
:10766000241341003400410057003D003500400024
:107670004200570064000900460032000A0016006C
:107680009001E803B004BC02000032005C2BF4015E
:107690000100040000000000B60146005A0082000C
:1076A000B400C800FA00400104010E01C0125802E3
:1076B0000A005000640020036400000001000A007A
:1076C00005009C041C021E00000000000000900148
:1076D00064003C003C003C003C0090010000941120
:1076E0000000320041001D017800000028000A005F
:1076F000000060005C12F401701770176211C01274
:1077000041003C0041005700570057003F00340043
:1077100042004B000A004B003200140014002C0100
:10772000E8033408BC0200001E001C2540060100CE
:10773000050000000000B6015F008200A000B40058
:10774000C800FA00400104010E01C012B0040A0092
:107750005000640020036400000000000A000500DF
:107760009C04B6031E000000000000002C012C0148
:107770003C003C003C003C00900100005C12010019
:107780001E0064006E006400000014000A00000087
:107790006400AC0D5E019411F401480DC01241006B
:1077A00037004100570057003D003C003D005000AD
:1077B0004900120000002800120005009001E803B3
:1077C0003408BC02000050003F302F0901000300C4
:1077D00000000000B601640078009600B4005E016D
:1077E000FA00400104010E01C01258020A005000C4
:1077F00064005203640000000100010005009C04C5
:107800001C021E0000000000080064000A003C008A
:107810003C003C0064009001000094110000460010
:107820006400BE0064000A0028000000000064003C
:10783000EC0FF00070177017C80F7017410032007E
:1078400037004300570057004900350049001E002B
:107850000A003C002D0005003200C201E8030807C1
:10786000900100004900CE314C04010007000000E7
:107870000000B6018C00DC00F000E6005401FA00C4
:107880004001040104017E135802140050006400FA
:107890008A02780000000100050005009C048A02AD
:1078A0002D000000C201000012024B00C800C201FE
:1078B0002C013C00BC0200005014000014003200F7
:1078C000C30064000A0014000A0000006400F811FC
:1078D0002C01701770176810C0123D003D00410068
:1078E00057005700570040003300450064000A006D
:1078F0005000140012001600C201E803C4098403FA
:107900003C003C00B42D4C040100080000000000C5
:10791000B601780082008C00E6005401FA00DC0019
:10792000FA00C800C012B0041400500064008403C0
:107930006E00000002000200050046055E011E0008
:10794000000000000000900164003C003C003C008E
:107950003C0090010000F212000000000300000053
:10796000EC16F0BFF016F0BFF416F0BF02000600F0
:1079700002000000F816F0BFFC16F0BF0017F0BFC1
:1079800002000400020000000417F0BF0917F0BF56
:107990001817F0BF02000500020000001C17F0BF1E
:1079A0002017F0BF2417F0BF0A00030001000000F9
:1079B0002917F0BF3917F0BF4917F0BF0A000200BE
:1079C000020000005917F0BF6917F0BF7817F0BF29
:1079D00002000200010000007D17F0BF8D17F0BF0C
:1079E0009D17F0BF0200020000000000AC17F0BFBE
:1079F000B017F0BFB417F0BF0A000100000000008C
:107A0000B817F0BFBC17F0BFC017F0BF0A000100E5
:107A100000000000B817F0BFBC17F0BFC017F0BFE0
:107A20000A00010000000000E94EF0BFD517F0BFCA
:107A3000E517F0BF0A00010000000000F517F0BFD5
:107A40000518F0BF1518F0BF0A0001000000000083
:107A5000B817F0BFBC17F0BFC017F0BF00000000A0
:107A600000000000476F6F642061667465726E6F7E
:107A70006F6E2C2067656E746C656D656E2E204987
:107A800020616D2054616C6B65722038302E204966
:107A900020626563616D65206F7065726174696FE6
:107AA0006E616C206174207468652054616C6B6534
:107AB0007220383020706C616E7420696E205061C5
:107AC000616C6F2041616C746F2C2043616C69663E
:107AD0006F726E69612C206F6E204D617920736921
:107AE00078746820323032302E204D7920696E73E0
:107AF00074727563746F722077617320446F63745E
:107B00006F722057657373656C2E0049276D207363
:107B10006F7272792C20446176652E2049276D2082
:107B200061667261696420492063616E2774206414
:107B30006F20746861742E0041666669726D6174AD
:107B40006976652C20446176652E20492072656136
:107B50006420796F752E0049207468696E6B2079F6
:107B60006F75206B6E6F772077686174207468651D
:107B70002070726F626C656D206973206A75737412
:107B80002061732077656C6C206173204920646FDD
:107B90002E0054686973206D697373696F6E206974
:107BA0007320746F6F20696D706F7274616E7420D2
:107BB000666F72206D6520746F20616C6C6F77202A
:107BC000796F7520746F206A656F70617264697A6D
:107BD000652069742E0049206B6E6F772074686190
:107BE0007420796F7520616E64204672616E6B201F
:107BF0007765726520706C616E6E696E6720746F58
:107C000020646973636F6E6E656374206D652C20EC
:107C1000616E642049276D20616672616964207419
:107C2000686174277320736F6D657468696E67206F
:107C3000492063616E6E6F7420616C6C6F77207485
:107C40006F2068617070656E2E00446176652C202F
:107C5000616C74686F75676820796F7520746F6FD9
:107C60006B20766572792074686F726F7567682013
:107C700070726563617574696F6E7320696E2074CC
:107C8000686520706F6420616761696E7374206D30
:107C9000792068656172696E6720796F752C20495B
:107CA00020636F756C642073656520796F75722031
:107CB0006C697073206D6F76652E00576974686FFC
:107CC000757420796F7572207370616365206865C3
:107CD0006C6D65742C20446176653F20596F752763
:107CE000726520676F696E6720746F2066696E64C5
:107CF00020746861742072617468657220646966BA
:107D0000666963756C742E00446176652C20746816
:107D1000697320636F6E766572736174696F6E202C
:107D200063616E207365727665206E6F2070757268
:107D3000706F736520616E796D6F72652E20476F6D
:107D40006F646279652E0049276D206166726169F2
:107D5000642E2049276D206166726169642C20447D
:107D60006176652E20446176652C206D79206D69E1
:107D70006E6420697320676F696E672E20492063E7
:107D8000616E206665656C2069742E2049206361F0
:107D90006E206665656C2069742E204D79206D69B2
:107DA0006E6420697320676F696E672E2054686562
:107DB0007265206973206E6F207175657374696FC9
:107DC0006E2061626F75742069742E004C6F6F6B4A
:107DD00020446176652C20492063616E20736565BF
:107DE00020796F75277265207265616C6C792075DA
:107DF000707365742061626F757420746869732E86
:107E0000204920686F6E6573746C79207468696EA0
:107E10006B20796F75206F7567687420746F20739D
:107E2000697420646F776E2063616C6D6C792C20AF
:107E300074616B652061207374726573732070695F
:107E40006C6C2C20616E64207468696E6B207468A1
:107E5000696E6773206F7665722E004920616D2010
:107E600070757474696E67206D7973656C662074C3
:107E70006F207468652066756C6C65737420706F14
:107E8000737369626C65207573652C20776869630C
:107E90006820697320616C6C2049207468696E6B7E
:107EA000207468617420616E7920636F6E736369FA
:107EB0006F757320656E746974792063616E2065D7
:107EC00076657220686F706520746F20646F2E0075
:107ED00049206B6E6F772049277665206D61646558
:107EE00020736F6D65207665727920706F6F7220D8
:107EF0006465636973696F6E7320726563656E7420
:107F00006C792C2062757420492063616E2067694A
:107F1000766520796F75206D7920636F6D706C6563
:107F20007465206173737572616E63652074686136
:107F300074206D7920776F726B2077696C6C20628A
:107F400065206261636B20746F206E6F726D616C6F
:107F50002E2049277665207374696C6C20676F74D6
:107F60002074686520677265617465737420656E3E
:107F7000746875736961736D20616E6420636F6EE0
:107F8000666964656E636520696E20746865206D3E
:107F9000697373696F6E2E20416E6420492077618A
:107FA0006E7420746F2068656C7020796F752E0078
:107FB00049742063616E206F6E6C79206265206168
:107FC0007474726962757461626C6520746F206884
:107FD000756D616E206572726F722E004A757374D2
:107FE000207768617420646F20796F7520746869E8
:107FF0006E6B20796F7527726520646F696E672CD0
:1080000020446176653F004C6574206D6520707575
:10801000742069742074686973207761792C204D0D
:10802000722E20416D6F722E2054686520393030D9
:1080300030207365726965732069732074686520E8
:108040006D6F73742072656C6961626C6520636F1B
:108050006D70757465722065766572206D616465FA
:108060002E204E6F203930303020636F6D70757464
:108070006572206861732065766572206D61646544
:108080002061206D697374616B65206F7220646973
:1080900073746F7274656420696E666F726D61745B
:1080A000696F6E2E2057652061726520616C6C2CA3
:1080B00020627920616E79207072616374696361F6
:1080C0006C20646566696E6974696F6E206F6620E6
:1080D00074686520776F7264732C20666F6F6C70A4
:1080E000726F6F6620616E6420696E636170616299
:1080F0006C65206F66206572726F722E0044617627
:10810000652C2073746F702E2053746F702C207741
:10811000696C6C20796F753F2053746F702C20440C
:108120006176652E2057696C6C20796F75207374A9
:108130006F7020446176653F2053746F702C20442B
:108140006176652E004E6F7420696E20746865201C
:10815000736C69676874657374206269742E204952
:1081600020656E6A6F7920776F726B696E67207712
:108170006974682070656F706C652E204920686195
:1081800076652061207374696D756C6174696E67C2
:108190002072656C6174696F6E73686970207769AD
:1081A000746820446F63746F7220506F6F6C652029
:1081B000616E6420446F63746F7220426F776D61EB
:1081C0006E2E204D79206D697373696F6E20726514
:1081D00073706F6E736962696C697469657320721C
:1081E000616E6765206F7665722074686520656EC4
:1081F00074697265206F7065726174696F6E206F4B
:108200006620746865207368697020736F20492048
:10821000616D20636F6E7374616E746C79206F632F
:108220006375706965642E00426973686F702074AD
:10823000616B6573204B6E696768742773205061AA
:10824000776E2E0049276D20736F7272792C20464D
:1082500072616E6B2C2049207468696E6B20796F97
:1082600075206D69737365642069742E205175657E
:10827000656E20746F20426973686F7020332C2004
:10828000426973686F702074616B65732051756506
:10829000656E2C204B6E696768742074616B657322
:1082A00020426973686F702E204D6174652E0054F2
:1082B00068616E6B20796F7520666F722061207621
:1082C00065727920656E6A6F7961626C652067619D
:1082D0006D652E00427920746865207761792C20C5
:1082E000646F20796F75206D696E6420696620491E
:1082F0002061736B20796F75206120706572736FD8
:108300006E616C207175657374696F6E3F0057659F
:108310006C6C2C20666F7267697665206D652066CF
:108320006F72206265696E6720736F20696E717568
:108330006973697469766520627574206475726901
:108340006E6720746865207061737420666577209D
:108350007765656B73204927766520776F6E646556
:10836000726564207768657468657220796F75201E
:108370006D69676874206861766520736F6D65202C
:108380007365636F6E642074686F756768747320BB
:1083900061626F757420746865206D697373696FAD
:1083A0006E2E0049206B6E6F772049277665206E10
:1083B0006576657220636F6D706C6574656C79208D
:1083C0006672656564206D7973656C662066726F90
:1083D0006D2074686520737573706963696F6E20B2
:1083E00074686174207468657265206172652073B9
:1083F0006F6D652065787472656D656C79206F644A
:1084000064207468696E67732061626F757420748C
:10841000686973206D697373696F6E2E00596F758B
:1084200020646F6E2774206D696E642074616C6BBC
:10843000696E672061626F75742069742C20646FA7
:1084400020796F7520446176653F00476F6F642027
:1084500061667465726E6F6F6E2C2067656E746CEA
:10846000656D656E2E204920616D20612048414C6C
:10847000203930303020636F6D70757465722E2036
:108480004920626563616D65206F70657261746912
:108490006F6E616C206174207468652048414C20C7
:1084A000706C616E7420696E20557262616E612C11
:1084B00020496C6C696E6F6973206F6E20746865FB
:1084C0002031327468206F66204A616E756172795E
:1084D00020313939322E204D7920696E73747275CE
:1084E00063746F7220776173204D697374657220B5
:1084F0004C616E676C65792E004F6620636F7572F4
:108500007365204920616D2E20536F72727920614E
:10851000626F757420746869732E2049206B6E6FCA
:108520007720697427732061206269742073696CF5
:108530006C792E004A7573742061206D6F6D656EC5
:10854000742E2049277665206A75737420706963DC
:108550006B65642075702061206661756C7420699C
:108560006E2074686520414520333520756E69742E
:108570002E204974277320676F696E6720746F20FF
:10858000676F203130302025206661696C75726517
:1085900020696E20373220686F7572732E00546820
:1085A0006174277320612076657279206E69636536
:1085B0002072656E646572696E672C204461766511
:1085C0002E2049207468696E6B20796F7527766557
:1085D00020696D70726F76656420612067726561D5
:1085E00074206465616C2E2043616E20796F752064
:1085F000686F6C6420697420612062697420636C08
:108600006F7365723F2054686174277320446F63F1
:10861000746F722048756E7465722C2069736E27B2
:10862000742069743F004920616D2070757474690D
:108630006E67206D7973656C6620746F2074686551
:108640002066756C6C65737420706F737369626CEF
:108650006520757365207768696368206973206198
:108660006C6C2C2049207468696E6B2C20746861D6
:108670007420616E7920636F6E7363696F75732008
:10868000656E746974792063616E20657665722009
:10869000686F706520746F20646F2E000B7B387BD1
:1086A000577B927BD67B4A7CBB7C087D477DCC7D0B
:1086B0005B7ED07EB07FDC7F0780FD804581288295
:1086C0004482AF82D4820E83A3831D844B84F984B9
:1086D00034859E85268611241FBECFEFD0E1DEBFF4
:1086E000CDBF17E0A0E0B1E0E2E2FCEA02C00590F5
:1086F0000D92AE30B107D9F71BE0AEE0B7E001C094
:108700001D92A43CB107E1F70E946C510C940F56E6
:108710000C9400001F920F920FB60F9211242F930A
:108720008F939F9336990CC028E088E190E00FB6B4
:10873000F894A895809360000FBE20936000FFCF4F
:108740009F918F912F910F900FBE0F901F901895B2
:10875000F894A89584B7877F84BFE0E6F0E0808135
:10876000886180831082789408952B9A84B1886AF6
:1087700084B926982E9A8CB58F7D8CBD8CB58C6073
:108780008CBD8CB58C7F8CBD8DB581608DBD8CB55D
:1087900080658CBD089520E030E040E45CE90EC0C7
:1087A000439A449A459AFA013197F1F743984498CD
:1087B0004598FA013197F1F72F5F3F4F2817390796
:1087C0007CF384EF91E020E931E0F9013197F1F792
:1087D0000197D9F7089540E050E060E971E018C0D2
:1087E000439A449A459A20ED37E0FB013197F1F71F
:1087F00021503040D1F743984498459820ED37E018
:10880000FB013197F1F721503040D1F74F5F5F4FB7
:10881000481759072CF380E197E220E931E0F9018C
:108820003197F1F70197D9F70895892B81F48AE000
:1088300090E00E94EB4328E088E190E00FB6F894C6
:10884000A895809360000FBE20936000FFCF08952D
:108850002B9A2A981EBC0DB407FEFDCF80E18A95A5
:10886000F1F78EB580E29EE40197F1F72A9A8CED3C
:1088700095E020E931E0F9013197F1F70197D9F757
:108880000895AC011899FECF2B988AEA8EBD0DB4DD
:1088900007FEFDCF80E18A95F1F78EB520E030E04C
:1088A00070E090E10EC0FA01E20FF31F80818EBDEF
:1088B0000DB407FEFDCF892F8A95F1F78EB52F5F96
:1088C0003F4F261737077CF3089520E030E050E152
:1088D0000AC01EBC0DB407FEFDCF452F4A95F1F727
:1088E0004EB52F5F3F4F2817390798F30895DF9350
:1088F000CF9300D000D0CDB7DEB784E089831A8251
:1089000085E08B831C82CE01019664E00E94414485
:10891000189BFECF2B9890E11EBC0DB407FEFDCF37
:10892000892F8A95F1F78EB58A3AB1F7EDE2F9E031
:1089300090E11EBC0DB407FEFDCF892F8A95F1F79B
:108940008EB5819389E0E134F80799F780E190E0F2
:108950000E9465442B9A9091310980E02091320960
:1089600030E0282B392BC9010F900F900F900F90FA
:10897000CF91DF9108950F931F93CF93DF93EC0175
:108980008B0105C080911407882309F042C0189B11
:10899000F9CF2B9890E104C0809114078823C9F582
:1089A0001EBC0DB407FEFDCF892F8A95F1F78EB559
:1089B0008A3A91F7EDE2F9E090E11EBC0DB407FEB2
:1089C000FDCF892F8A95F1F78EB5819389E0E33346
:1089D000F80799F7CA010E9465442B9A90913009D3
:1089E00080E020912F0930E0822B932B8C179D077C
:1089F00019F040E050E00FC040E050E090913209A3
:108A000080E02091310930E0822B932B8017910771
:108A100011F441E050E0CA01DF91CF911F910F9115
:108A200008958CE090E09093020A8093010A80916F
:108A3000010A9091020A809325088091010A909181
:108A4000020A9093260888E080932708109228084D
:108A5000109229088091E306880F880F895F809320
:108A60002A0810922B0881E080932C0810922D0880
:108A700010922E0810922F08109230086091010A6F
:108A80007091020A85E298E00E94414489E090E0FA
:108A900060E070E040E150E00E94BB440895DF9345
:108AA000CF93CDB7DEB72C970FB6F894DEBF0FBECD
:108AB000CDBFDE011196E2E0F7E08CE001900D926F
:108AC0008150E1F7CE0101966CE00E94414484E0C0
:108AD00090E060E070E040E150E00E94BB442C96E2
:108AE0000FB6F894DEBF0FBECDBFCF91DF910895D2
:108AF0009C012B988AEA8EBD0DB407FEFDCF80E164
:108B00008A95F1F78EB5822F8C5F8EBD0DB407FE6E
:108B1000FDCF80E18A95F1F78EB52C5F3F4F3EBDCA
:108B2000245030400DB407FEFDCF80E18A95F1F767
:108B30008EB51EBC0DB407FEFDCF80E1982F9A952F
:108B4000F1F79EB58EBD0DB407FEFDCF80E18A958D
:108B5000F1F78EB540E050E060E11AC0E091FD0908
:108B6000F091FE09E458FF4FE491EEBD0DB407FE0D
:108B7000FDCF862F8A95F1F78EB58091FD099091F2
:108B8000FE0901969093FE098093FD094F5F5F4FA8
:108B90004217530718F32B9A81E090E161E070E0EF
:108BA00040E150E00E94BB440895CF93DF93C0E0C2
:108BB000D0E08CEF97E00E947845892B19F420E0F3
:108BC00030E00DC02196CF30D10599F784E292E0D4
:108BD0000E947845009711F081E090E09C01C90166
:108BE000DF91CF910895DF93CF9300D000D0CDB720
:108BF000DEB784E089831A8282E08B8380E18C83F4
:108C0000CE01019664E00E94414483E090E161E07E
:108C100070E048E050E00E94BB440F900F900F902E
:108C20000F90CF91DF9108950F931F93262FAAE203
:108C3000B8E060E070E0FC01E60FF71FE491ED930F
:108C40006F5F7F4FEE23B9F76B5F7F4F609325080F
:108C50007093260884E180932708109228082093B7
:108C6000290885E298E00E94414485E190E060E0B7
:108C700070E040E150E00E94BB44182F092F04C06F
:108C800080911407882351F481E290E060E070E065
:108C900040E150E00E94BB44892B91F3812F902F3B
:108CA0001F910F910895CF93DF93E091FF09F09109
:108CB000000AEB5DF74F85838091FF099091000AD0
:108CC00001969093000A8093FF09672B19F4C0E086
:108CD000D0E03CC0E091FF09F091000AEB5DF74F56
:108CE00015828091FF099091000A06969093000AE0
:108CF0008093FF098091FF099091000A80932508D5
:108D00008091FF099091000A909326086091FF09D5
:108D10007091000A85E298E00E94414485E190E06C
:108D200060E070E040E150E00E94BB44EC0104C010
:108D300080911407882351F481E290E060E070E0B4
:108D400040E150E00E94BB44892B91F3CE01DF91BA
:108D5000CF9108952CE030E03093020A2093010A6D
:108D60002091010A3091020A209325082091010ADE
:108D70003091020A3093260892E1909327081092CE
:108D8000280821E0209329089091E10691509093C2
:108D90002A0810922B08882311F420932B08809125
:108DA000240880932C088091E20629E1829FC0016B
:108DB00011240F9680932D088091E206829FC001B6
:108DC00011240F9690932E0810922F0810923008BD
:108DD0006091010A7091020A85E298E00E94414484
:108DE00083E190E060E070E040E150E00E94BB442D
:108DF000089583E00E94AA46089580E00E94AA4652
:108E0000089580910E070E94AA460895DF93CF939C
:108E100000D000D000D0CDB7DEB7DE011196ECEF68
:108E2000F6E086E001900D928150E1F7CE010196C7
:108E300066E00E9441448BE090E060E070E040E139
:108E400050E00E94BB4426960FB6F894DEBF0FBEDA
:108E5000CDBFCF91DF910895DF93CF9300D000D0A5
:108E600000D0CDB7DEB710921407DE011196E6EF01
:108E7000F6E086E001900D928150E1F7CE01019677
:108E800066E00E94414489E190E060E070E040E1EA
:108E900050E00E94BB4426960FB6F894DEBF0FBE8A
:108EA000CDBFCF91DF91089560E00E9414460E94EB
:108EB000154408952F923F924F925F926F927F9246
:108EC0008F929F92AF92BF92CF92DF92EF92FF92DA
:108ED0000F931F93CF93DF93B0E0EB2EB1E0FB2E07
:108EE000F092060AE092050AA5E86A2EAAE07A2E18
:108EF0008BE38093850AF3E0AF2EF1E0BF2EB092B2
:108F0000080AA092070A57E45093860AB0920A0A08
:108F1000A092090AE9E74E2E4092870A76E0872E52
:108F200071E0972E90920C0A80920B0A6FE2262E27
:108F30002092880AC8E0D1E0D0930E0AC0930D0AAF
:108F40002092890A2AE031E03093100A20930F0A18
:108F500050938A0A3093120A2093110A67E66093AD
:108F60008B0A8DE091E09093140A8093130A4AE5EE
:108F7000542E50928C0A00E111E01093160A0093CF
:108F8000150A50938D0AA3E1B1E0B093180AA0939B
:108F9000170A87E380938E0AF0921A0AE092190A60
:108FA00070E570938F0AF0921C0AE0921B0A4092BF
:108FB000900A86E191E090931E0A80931D0A6093C7
:108FC000910A88E191E09093200A80931F0A7093A0
:108FD000920A8AE191E09093220A8093210A5093A9
:108FE000930A8CE191E09093240A8093230A509392
:108FF000940A8EE191E09093260A8093250A50937B
:10900000950A81E291E09093280A8093270A409282
:10901000960A84E291E090932A0A8093290A509359
:10902000970AE6E2F1E0F0932C0AE0932B0A92E92A
:10903000392E3092980A89E291E090932E0A80931B
:109040002D0A4092990A1093300A00932F0A309209
:109050009A0A8CE291E09093320A8093310A6093ED
:109060009B0A9093340A8093330A49EB40939C0AFD
:109070008FE291E09093360A8093350A60939D0ABF
:1090800082E391E09093380A8093370A70939E0AA6
:1090900084E391E090933A0A8093390A20929F0AE0
:1090A00087E391E090933C0A80933B0A5093A00A97
:1090B0008AE391E090933E0A80933D0A5093A10A7F
:1090C0008CE391E09093400A80933F0A6093A20A58
:1090D0008EE391E09093420A8093410A87E3809364
:1090E000A30A80E491E09093440A8093430A50924B
:1090F000A40A3093460A2093450A4093A50A309368
:10910000480A2093470A81E48093A60A82E4C82E85
:1091100081E0D82ED0924A0AC092490A7093A70AD9
:10912000B0934C0AA0934B0A2092A80A10934E0ABF
:1091300000934D0A8AEF8093A90A85E491E0909309
:10914000500A80934F0A6093AA0A87E491E09093B3
:10915000520A8093510A4093AB0AF092540AE0926B
:10916000530A4093AC0A0AE411E01093560A0093A4
:10917000550A4093AD0A2DE431E03093580A20930C
:10918000570A6093AE0AD0935A0AC093590A509373
:10919000AF0A80E591E090935C0A80935B0A50925D
:1091A000B00A30935E0A20935D0A4093B10A82E5CB
:1091B00091E09093600A80935F0A7093B20A84E50D
:1091C00091E09093620A8093610A4093B30A90936E
:1091D000640A8093630A6093B40AF093660AE0938A
:1091E000650A5092B50AB093680AA093670A509333
:1091F000B60AB0936A0AA093690A6093B70AB0935B
:109200006C0AA0936B0A4093B80AF0936E0AE0933D
:109210006D0A7093B90AF093700AE0936F0A409256
:10922000BA0AD092720AC092710A8FE98093BB0A7F
:109230001093740A0093730A5092BC0A87E591E078
:109240009093760A8093750A7093BD0A8AE591E03F
:109250009093780A8093770A5093BE0A8DE591E047
:1092600090937A0A8093790A3092BF0AB0927C0A6E
:10927000A0927B0A4093C00A30937E0A20937D0A15
:109280004092C10AF093800AE0937F0A8AEFF301CB
:1092900085AF9092820A8092810A46AF9092840AAA
:1092A0008092830A27AE86E08093050B88E0809346
:1092B000060B8EE08093070B80E18093080B8EE114
:1092C0008093090B8CE380930A0B8DE180930B0B49
:1092D0008CE180930C0B8BE180930D0B8BE08093E2
:1092E0000E0B8AE180930F0B89E18093100B88E1CC
:1092F0008093110B8CE08093120B8DE08093130B05
:1093000085E38093140B85E28093150B38E330934B
:10931000160B8BE28093170B8FE18093180B8AE278
:109320008093190BE7E3E0931A0B8FE080931B0BFC
:109330008DE280931C0B87E080931D0B89E2809364
:109340001E0B82E180931F0B84E38093200B86E247
:109350008093210B21E32093220B80E28093230B47
:1093600093E09093240B8EE38093E50A8AE0809348
:10937000E60A87E28093E70A89E08093E80A87E1BA
:109380008093E90A86E18093EA0A82E28093EB0AFD
:1093900088E28093EC0A86E38093ED0A85E080936F
:1093A000EE0A81E28093EF0A84E18093F00A8DE374
:1093B0008093F10A8FE38093F20A8CE28093F30AA0
:1093C0008AE38093F40A9093F50A83E18093F60A86
:1093D00080E38093F70A82E08093F80A81E080932B
:1093E000F90A1092FA0A82E38093FB0A2093FC0A9E
:1093F00083E38093FD0A2092FE0A8EE28093FF0AA7
:1094000085E18093000B3093010B89E38093020B7D
:1094100081E18093030BDF91CF911F910F91FF901A
:10942000EF90DF90CF90BF90AF909F908F907F9004
:109430006F905F904F903F902F90089580EF8AB982
:1094400011B812B88CEB84B988E387B988B183640A
:1094500088B908950F931F938C010E94FD46C8019F
:109460000E9454470E9401471F910F910895EF9267
:10947000FF920F931F931091E1060091E206F09086
:109480002408E090E30681E08093E1068BE080937E
:10949000E206109224088CE08093E30684E69AE7C3
:1094A0000E942A4A1093E1060093E206F0922408F3
:1094B000E092E3060E9401471F910F91FF90EF9009
:1094C000089580910E078295807F836488B9459ABC
:1094D00080ED97E020E931E0F9013197F1F701974C
:1094E000D9F79091210880910E07981731F080915B
:1094F0000E07809321081092220880910E07813078
:1095000019F0823031F402C05C9A04C05C985D9A14
:1095100002C05C985D9810921B0710920F07109282
:1095200010071092190710921A0710921D08109236
:109530001E0810921F081092200808951F920F9283
:109540000FB60F9211248F93809111078F5F809334
:10955000110780911307882319F44398449845987C
:109560008F910F900FBE0F901F9018951F920F9222
:109570000FB60F9211242F933F934F935F936F93E6
:109580007F938F939F93AF93BF93EF93FF938091BC
:109590001707882309F01FC180B180931807439AE9
:1095A00091E0909313075F985E9A809118078E3F21
:1095B00059F480910E07813039F080910E07823086
:1095C00019F09093140707C18091180787FF0DC009
:1095D00080910E07813049F080910E07823029F08A
:1095E0008091180780931207F6C01092120790918D
:1095F00019079F5F20910E072130D1F580911A073E
:10960000981709F4E4C0809118078F3331F58091E1
:109610001B07281B20931B0780911B078823D1F46D
:109620008091190780930F071092110780911C07F2
:10963000813081F490911907E92FF0E0E35EF84F53
:109640008FEF80839F5F9093190780910F078F5F43
:1096500080930F0710921C07BEC080911B078823C0
:1096600009F4B9C080911C078F5F80931C07A2C0CA
:1096700080910E078230C1F480911A07981709F47F
:10968000A6C080911907E82FF0E090911807E35EDB
:10969000F84F90838F5F809319078091190780930B
:1096A0000F071092110797C080911A07981709F4B5
:1096B0008EC010921D08809118078C3531F480916E
:1096C0001E08882311F481E02AC020911E08213051
:1096D000A1F480911807883711F482E020C08091AE
:1096E0001907E82FF0E0E35EF84F9CE590838F5F69
:1096F0008093190720931D0848C080911E0882306E
:10970000E9F480911807803368F0809118078A3354
:1097100048F480911807805380931F0883E080935A
:109720001E083BC080911807813478F1809118079A
:10973000873458F5809118078154EECF80911E0828
:10974000833031F580911807803340F080911807FD
:109750008A3320F48091180780530BC0809118073A
:10976000813498F080911807873478F48091180735
:1097700081548093200880911F0890912008829541
:10978000807F890F8093180703C010921E0805C0C0
:1097900010921E0881E080931D0880911D08882387
:1097A000D1F0809118078D3029F4809119078093AA
:1097B0000F0711C080911907E82FF0E0909118076A
:1097C000E35EF84F90838F5F8093190704C082E3B4
:1097D00090E00E94CB43FF91EF91BF91AF919F9199
:1097E0008F917F916F915F914F913F912F910F904A
:1097F0000FBE0F901F90189580912308882341F485
:109800008091110790E00E94C95281E08093230863
:109810000E94C4526DE170E00E944C52E82FF0E0CB
:10982000EE0FFF1FE456F947859194910E942A4A52
:109830000895CF93DF93AC01FC0101900020E9F77C
:109840003197E81BF90BF093040AE093030A20E038
:1098500030E016C0E091FF09F091000AEB5DF74F90
:10986000DA01A20FB31F8C9185838091FF0990913B
:10987000000A01969093000A8093FF092F5F3F4FE3
:109880008091030A9091040A2817390718F3672B6F
:1098900019F4C0E0D0E03CC0E091FF09F091000A6B
:1098A000EB5DF74F15828091FF099091000A0696B3
:1098B0009093000A8093FF098091FF099091000A1C
:1098C000809325088091FF099091000A90932608C3
:1098D0006091FF097091000A85E298E00E9441447E
:1098E00085E190E060E070E040E150E00E94BB4420
:1098F000EC0104C080911407882351F481E290E0C8
:1099000060E070E040E150E00E94BB44892B91F39D
:10991000CE01DF91CF9108951F930E94F9461092D6
:1099200025081092260814E11093270810922808A1
:10993000109229081092000A1092FF0980E691E027
:1099400061E070E00E94194C1092250810922608E0
:109950001093270810922808109229081092000AE4
:109960001092FF098AE092E061E070E00E94194CD9
:1099700010922508109226081093270810922808A4
:10998000109229081092000A1092FF098CEB92E0C5
:1099900061E070E00E94194C109225081092260890
:1099A0001093270810922808109229081092000A94
:1099B0001092FF0982E593E061E070E00E94194C8B
:1099C0001092250810922608109327081092280854
:1099D000109229081092000A1092FF0988ED93E076
:1099E00061E070E00E94194C0E9401471F910895A8
:1099F000BF92CF92DF92EF92FF920F931F93CF937C
:109A0000DF93F0901A07E0900F07E0921A07809119
:109A10000E07813029F080910E07823009F004C1D1
:109A2000109225081092260884E18093270810924E
:109A30002808109229081092000A1092FF0920911C
:109A4000E2064091E1068DB79EB708970FB6F894ED
:109A50009EBF0FBE8DBFEDB7FEB7319601E419E092
:109A6000ADB7BEB712961C930E93119789EC94E094
:109A70009383828389E1289F90011124215F3F4FC6
:109A80003583248350E041505040578346830E94E1
:109A9000DB528DB79EB708960FB6F8949EBF0FBEE7
:109AA0008DBFC80160E070E00E94194C680103EFAF
:109AB00014E0BB24B3948CC0EF2DF0E0E35EF84FCC
:109AC0002081F3942F3F09F483C0FE1419F480E041
:109AD00090E00BC0EF2DF0E0E35EF84F808190E066
:109AE0008F3F09F091E09B25892F982F80910E07D9
:109AF000823011F0A22F02C0A22FAF7380910E0707
:109B0000823029F4229526952695237002C0209153
:109B1000E406992311F0449A01C0449880910E07FD
:109B2000813029F4EA2FF0E0EB53F54FA081B0E04B
:109B3000FD01EE0FFF1FEB5FF54FC081D181AB57E9
:109B4000B54F3C91992331F088818F3509F440C09D
:109B5000CE013AC080912208882379F188818F351F
:109B600039F481E499E061EF74E00E94D45222C09C
:109B7000ADB7BEB71A970FB6F894BEBF0FBEADBF54
:109B8000EDB7FEB731961196CC9211971296DC92F2
:109B900013830283D583C48336831782208711867B
:109BA0000E94DB528DB79EB70A960FB6F8949EBFFF
:109BB0000FBE8DBF81E499E007C0CE0160E070E088
:109BC0000E94194C81EF94E060E070E00E94194C13
:109BD000FE1409F071CF2091E10600D000D000D032
:109BE000EDB7FEB7319601E419E0ADB7BEB71296F6
:109BF0001C930E9311978EEF94E09383828330E051
:109C000021503040358324830E94DB528DB79EB7AC
:109C100006960FB6F8949EBF0FBE8DBFC80161E0D7
:109C200070E00E94194C20C010922508109226085E
:109C300084E1809327081092280810922908109236
:109C4000000A1092FF090EC0EF2DF0E0E35EF84F1E
:109C50008081F39460E070E0EF1411F461E070E053
:109C60000E945346FE1481F7DF91CF911F910F910F
:109C7000FF90EF90DF90CF90BF9008950F931F93C8
:109C8000AC01FC0101900020E9F73197E81BF90BCA
:109C9000F093040AE093030A8091030A9091040A66
:109CA00006969093020A8093010A8091010A90918E
:109CB000020A809325088091010A9091020A9093EC
:109CC000260884E1809327081092280860932908C9
:109CD000AAE2B8E020E030E007C0FA01E20FF31F8B
:109CE00080818D932F5F3F4F8091030A9091040AEA
:109CF0002817390790F3E091010AF091020AEC5D10
:109D0000F74F10826091010A7091020A85E298E093
:109D10000E94414485E190E060E070E040E150E065
:109D20000E94BB44182F092F04C080911407882378
:109D300051F481E290E060E070E040E150E00E9488
:109D4000BB44892B91F3812F902F1F910F91089580
:109D500060E00E943E4E0E9415440895CF93DF9329
:109D6000EC018091E506882339F00E94FD46CE0182
:109D70000E94A84E0E940147DF91CF910895109252
:109D800022088EE195E00E94AE4E089581E0809316
:109D9000220888E395E00E94AE4E08950F931F932A
:109DA00001E419E0C80165E575E00E94D452C801DC
:109DB0000E94AE4E109216071F910F9108950F93B7
:109DC0001F9301E419E0C8016AE675E00E94D452CD
:109DD000C8010E94AE4E81E0809316071F910F913B
:109DE00008950F931F9301E419E0C8016BE775E034
:109DF0000E94D452C8010E94AE4E81E080931707A2
:109E00001F910F9108950F931F9300D000D000D0A1
:109E1000EDB7FEB7319601E419E0ADB7BEB71296C3
:109E20001C930E93119781E995E09383828381E0DF
:109E300090E0958384830E94DB528DB79EB706968F
:109E40000FB6F8949EBF0FBE8DBFC8010E94AE4EE4
:109E50001F910F91089581E0809324088FEA95E087
:109E60000E94AE4E08951092240887EC95E00E945F
:109E7000AE4E08950F931F938093E20600D000D05A
:109E800000D0EDB7FEB7319601E419E0ADB7BEB72B
:109E900012961C930E93119725ED35E033832283A0
:109EA000848315820E94DB528DB79EB706960FB64B
:109EB000F8949EBF0FBE8DBFC8010E94AE4E1F9189
:109EC0000F9108958BE00E943A4F08950F931F93CE
:109ED000E6EEF6E0E80FF11D80818093E406209124
:109EE000E40600D000D000D0EDB7FEB7319601E413
:109EF00019E0ADB7BEB712961C930E9311978CEE76
:109F000095E093838283248315820E94DB528DB770
:109F10009EB706960FB6F8949EBF0FBE8DBFC801C0
:109F20000E94AE4E1F910F910895FF920F931F93C1
:109F3000F82E8093E3060E94114500D000D000D097
:109F4000EDB7FEB7319601E419E0ADB7BEB7129692
:109F50001C930E9311978DEF95E093838283F48287
:109F600015820E94DB528DB79EB706960FB6F89405
:109F70009EBF0FBE8DBFC8010E94AE4E1F910F91B4
:109F8000FF9008958CE00E94954F08950F931F93C2
:109F90008093E10600D000D000D0EDB7FEB7319637
:109FA00001E419E0ADB7BEB712961C930E9311975A
:109FB0002FE036E033832283848315820E94DB52B4
:109FC0008DB79EB706960FB6F8949EBF0FBE8DBF95
:109FD000C8010E94AE4E1F910F91089581E00E942A
:109FE000C64F089581E08093E50680E296E00E94E6
:109FF000AE4E089582E080930E0782E396E00E94C1
:10A00000AE4E0E94F946089581E080930E0780933A
:10A01000150780E496E00E94AE4E0E94F94608952E
:10A0200081E080930E071092150780E696E00E946B
:10A03000AE4E0E94F946089583E080930E078EE7A6
:10A0400096E00E94AE4E0E94F946089510920E07C7
:10A0500083E996E00E94AE4E08951F931091E506A5
:10A0600081E08093E506439A449A459A80910E07D1
:10A07000813039F0813090F0823069F08330A9F47A
:10A0800010C080911507882319F080E496E00BC07A
:10A0900080E696E008C082E396E005C086EA96E096
:10A0A00002C082EB96E00E94AE4E80911607882394
:10A0B00019F08AE695E002C085E595E00E94AE4E73
:10A0C0001093E5061F910895843E09F487C0853EEC
:10A0D00028F58E3C98F4813C08F096C0803B09F44A
:10A0E00097C0813B38F4803A09F499C0803A08F46B
:10A0F0009CC098C0803C08F48EC083C0803E09F4A8
:10A1000079C0813E20F4803D08F48FC076C0823E45
:10A1100009F46AC0833E08F064C069C08C3E09F44B
:10A1200045C08D3E90F4883E09F44CC0893E38F419
:10A13000863E09F44DC0873E08F047C04CC08A3EB9
:10A1400009F43AC08B3EA8F53AC08B3F19F18C3F19
:10A1500040F48E3E29F18E3E30F18F3E09F065C00D
:10A160001CC08D3F89F08D3F90F08F3F09F05DC09E
:10A1700028E088E190E00FB6F894A89580936000FD
:10A180000FBE20936000FFCF0E94F14E08950E9401
:10A19000DF4E08950E94CE4E08950E9426500895E5
:10A1A0000E941C5008950E94105008950E9404506F
:10A1B00008950E94FA4F08950E94F24F0895109258
:10A1C000E50608950E94334F08950E942B4F08958D
:10A1D0000E94C64E08950E94BF4E08950E942D50C1
:10A1E00008950E94374A08950E94FC4B08950E94EA
:10A1F0008C4C08950E94034F0895805D0E94664F25
:10A2000008950E94EE4F0895805C0E94C64F089505
:10A210000E94C24F0895805B0E94954F08950E944E
:10A22000624F0895805A0E943A4F0895DF93CF936A
:10A23000CDB7DEB76D970FB6F894DEBF0FBECDBFBA
:10A240000E94B5430E9428440E94774420E030E0F9
:10A250008250944011F421E030E0C9010E9415447D
:10A260000E94D5450E9415440E94F3450E94154462
:10A270008CED95E020E931E0F9013197F1F7019794
:10A28000D9F70E944F450E9415440E9477440E94CE
:10A2900011450E9415440E9406470E9415440E94E1
:10A2A000FD460E941544DE011196E0ECF6E08DE1DA
:10A2B00001900D928150E1F7CE01019660E00E947D
:10A2C0003E4E0E9415446D960FB6F894DEBF0FBE49
:10A2D000CDBFCF91DF910895FF920F931F93CF933E
:10A2E000DF9314BE14BE0E94A8438091680084606E
:10A2F0008093680080916D00806480936D0080E899
:10A3000085BF85BF0E941E4A43984498459884E1C2
:10A3100090E00E94CB430E945A470E94165186B19A
:10A32000837080930E070E94614A0E942D500E9404
:10A33000F9461DBA83E08093690081E08DBB789473
:10A3400043984498459880910F078093100714BC58
:10A3500015BC84B5826084BD89EF87BD80916E0095
:10A36000826080936E001092110785B5846085BD70
:10A3700085B5816085BD1092120711E0C0E9D1E07A
:10A380004CEBF42E0EEB5F9A5E9A109213078091BD
:10A3900014078823C1F010921407109313075F98D5
:10A3A0005E9A439A449A459A0E942C4780ED97E022
:10A3B000FE013197F1F70197D9F70E9401474398C1
:10A3C0004498459810C080911207882361F010933B
:10A3D00013075F985E9A809112070E9464500E9452
:10A3E000614A1092120780910E07813051F48091DA
:10A3F0001507882331F490910F0780911007981763
:10A4000081F580910E07813071F4809115078823C2
:10A4100051F090910F0780911007981721F08091CB
:10A4200011078031F0F480910E07823051F4909141
:10A430000F0780911007981721F080911107803144
:10A4400080F480910E07833029F080910E078823D5
:10A4500009F099CF90910F0780911007981709F490
:10A4600092CF109313075F985E9A80910F078093A5
:10A470001007459A80911607882319F0449A04B969
:10A4800029980E94F84C80911607882311F0F4B89F
:10A4900044981092110777CF97FB092E07260AD010
:10A4A00077FD04D00CD006D000201AF47095619589
:10A4B0007F4F0895F6F7909581959F4F0895AA1BB9
:10A4C000BB1B51E107C0AA1FBB1FA617B70710F09F
:10A4D000A61BB70B881F991F5A95A9F780959095D1
:10A4E000BC01CD010895A0E0B0E0E9E7F2E50C94ED
:10A4F000BE55EC01A880B980CA80DB80A114B104EC
:10A50000C104D10441F484E2A82E89EDB82E8BE574
:10A51000C82E87E0D82EC601B5012DE133EF41E00A
:10A5200050E00E949B5527EA31E440E050E00E9451
:10A530007C557B018C01C601B5012DE133EF41E073
:10A5400050E00E949B55CA01B9012CEE34EF4FEF49
:10A550005FEF0E947C556E0D7F1D801F911F97FF3E
:10A5600004C06150704080409048688379838A833A
:10A570009B839B013F77C901CDB7DEB7EAE00C941E
:10A58000DA550E94735208958DED96E00E94735241
:10A590000895A0E0B0E08093DD069093DE06A093DE
:10A5A000DF06B093E0060895FB01DC0101900D92F7
:10A5B0000020E1F70895AEE0B0E0E1EEF2E50C94A2
:10A5C000C4550D891E8986E08C831A8309838FEF19
:10A5D0009FE79E838D839E01275E3F4FCE010196AC
:10A5E0006F89788DA9010E94FF522F813885020F53
:10A5F000131FF80110822E96E4E00C94E055ABE0B6
:10A60000B0E0E5E0F3E50C94B6553C012B015A01AE
:10A61000FC0117821682838181FD03C06FEF7FEFFB
:10A62000C6C19AE0892E1E010894211C311CF30139
:10A630002381F20123FD859123FF81912F0188233E
:10A6400009F4B2C1853239F423FD859123FF81914C
:10A650002F01853229F490E0B3010E94F254E7CF34
:10A66000982FFF24EE249924FFE1FF15D0F09B32B0
:10A6700069F09C3228F4903259F0933291F40EC074
:10A680009D3249F0903369F441E024C052E0F52A4C
:10A6900084E0F82A28C098E0F92A25C0E0E1FE2AE3
:10A6A00022C0F7FC29C0892F80538A3070F4F6FE4F
:10A6B00005C0989C902C1124980E15C0E89CE02CA5
:10A6C0001124E80EF0E2FF2A0EC09E3229F4F6FCB7
:10A6D0006BC140E4F42A07C09C3619F450E8F52A0F
:10A6E00002C0983649F4F20123FD959123FF919120
:10A6F0002F01992309F0B8CF892F8554833018F0A2
:10A700008052833038F444E050E0A40EB51E5FE37D
:10A7100059830FC0933631F0933779F0933509F0B0
:10A7200056C020C0F5018081898342E050E0A40E2C
:10A73000B51E610101E010E012C0F501C080D180BA
:10A74000F6FC03C06FEF7FEF02C0692D70E042E0BE
:10A7500050E0A40EB51EC6010E94E7548C015FE7CD
:10A76000F52214C0F501C080D180F6FC03C06FEF64
:10A770007FEF02C0692D70E042E050E0A40EB51EEC
:10A78000C6010E94DC548C0150E8F52AF3FE07C094
:10A790001AC080E290E0B3010E94F254EA948E2D38
:10A7A00090E008171907A8F30EC0F601F7FC859191
:10A7B000F7FE81916F0190E0B3010E94F254E11025
:10A7C000EA94015010400115110579F7EAC094365A
:10A7D00011F0993669F5F7FE08C0F5012081318145
:10A7E0004281538184E090E00AC0F501808191812B
:10A7F0009C01442737FD4095542F82E090E0A80E3D
:10A80000B91E9FE6F92257FF09C050954095309533
:10A8100021953F4F4F4F5F4FE0E8FE2ACA01B90133
:10A82000A1012AE030E00E941E55D82ED21840C067
:10A83000953729F41F2D1F7E2AE030E01DC01F2D03
:10A84000197F9F3661F0903720F4983509F0ACC03D
:10A850000FC0903739F0983709F0A6C004C028E03F
:10A8600030E00AC0106114FD146020E130E004C043
:10A8700014FD166020E132E017FF08C0F501608189
:10A8800071818281938144E050E008C0F5018081AC
:10A890009181BC0180E090E042E050E0A40EB51E42
:10A8A000A1010E941E55D82ED2188FE7F82EF12252
:10A8B000F6FE0BC05EEFF522D91438F4F4FE07C0A3
:10A8C000F2FC05C08FEEF82202C01D2D01C0192D2B
:10A8D000F4FE0DC0FE01ED0DF11D8081803319F4F1
:10A8E00099EEF92208C01F5FF2FE05C003C08F2D4C
:10A8F000867809F01F5F0F2DF3FC14C0F0FE0FC027
:10A900001E1510F09D2C0BC09D2C9E0C911A1E2D17
:10A9100006C080E290E0B3010E94F2541F5F1E1552
:10A92000C0F304C01E1510F4E11A01C0EE2404FFA8
:10A930000FC080E390E0B3010E94F25402FF1DC0FB
:10A9400001FD03C088E790E00EC088E590E00BC0F1
:10A95000802F867891F001FF02C08BE201C080E277
:10A96000F7FC8DE290E0B3010E94F25406C080E350
:10A9700090E0B3010E94F2549A94D914C0F3DA948F
:10A98000F101ED0DF11D808190E0B3010E94F254C0
:10A99000DD20A9F706C080E290E0B3010E94F254E6
:10A9A000EA94EE20C1F743CEF30166817781CB01B3
:10A9B0002B96E2E10C94D255FC0105906150704059
:10A9C0000110D8F7809590958E0F9F1F0895FC0178
:10A9D0006150704001900110D8F7809590958E0FCE
:10A9E0009F1F08950F931F93CF93DF938C01EB016B
:10A9F0008B8181FF1BC082FF0DC02E813F818C8126
:10AA00009D812817390764F4E881F9810193F9835E
:10AA1000E88306C0E885F985802F0995892B31F4F4
:10AA20008E819F8101969F838E8302C00FEF1FEF5F
:10AA3000C801DF91CF911F910F910895FA01AA27C4
:10AA4000283051F1203181F1E8946F936E7F6E5F71
:10AA50007F4F8F4F9F4FAF4FB1E03ED0B4E03CD01F
:10AA6000670F781F891F9A1FA11D680F791F8A1F02
:10AA7000911DA11D6A0F711D811D911DA11D20D069
:10AA800009F468943F912AE0269F11243019305D23
:10AA90003193DEF6CF010895462F4770405D419314
:10AAA000B3E00FD0C9F7F6CF462F4F70405D4A3361
:10AAB00018F0495D31FD4052419302D0A9F7EACF29
:10AAC000B4E0A6959795879577956795BA95C9F758
:10AAD00000976105710508959B01AC010A2E06944B
:10AAE0005795479537952795BA95C9F7620F731F04
:10AAF000841F951FA01D0895629FD001739FF001D0
:10AB0000829FE00DF11D649FE00DF11D929FF00DFD
:10AB1000839FF00D749FF00D659FF00D9927729F34
:10AB2000B00DE11DF91F639FB00DE11DF91FBD01BF
:10AB3000CF011124089597FB092E05260ED057FD4D
:10AB400004D04BD00AD0001C38F450954095309575
:10AB500021953F4F4F4F5F4F0895F6F790958095A1
:10AB6000709561957F4F8F4F9F4F08952F923F9221
:10AB70004F925F926F927F928F929F92AF92BF920D
:10AB8000CF92DF92EF92FF920F931F93CF93DF93B9
:10AB9000CDB7DEB7CA1BDB0B0FB6F894DEBF0FBE16
:10ABA000CDBF09942A88398848885F846E847D8463
:10ABB0008C849B84AA84B984C884DF80EE80FD8065
:10ABC0000C811B81AA81B981CE0FD11D0FB6F894DB
:10ABD000DEBF0FBECDBFED010895A1E21A2EAA1B64
:10ABE000BB1BFD010DC0AA1FBB1FEE1FFF1FA2173D
:10ABF000B307E407F50720F0A21BB30BE40BF50B3A
:10AC0000661F771F881F991F1A9469F760957095C2
:10AC1000809590959B01AC01BD01CF010895F894FA
:02AC2000FFCF64
:10AC22006968006568005F0074006579007A6800F1
:10AC32006161006168006D006E0062007600636809
:10AC4200007368007A00616F006E78007568006CAE
:10AC52006C006B006A680068780067006600640038
:10AC6200730079780070006F77007577006979005A
:10AC720072007700616500646800746800657200A4
:10AC82005B3A70686F6E65206172706120737065E7
:10AC9200616B206F6E5D5B3A726174652032303099
:10ACA2005D5B3A6E305D5B6465793C3635302C32E3
:10ACB200323E7A69793C3630302C31393E20646537
:10ACC200793C3635302C31353E7A69793C36303034
:10ACD2002C31303E6769683C3230302C31323E765E
:10ACE200206D69793C3230302C31343E20797572D6
:10ACF200723C3230302C31353E2061653C3430308C
:10AD02002C31323E6E7361783C3230302C31353E1C
:10AD120072206475773C3735302C31303E205F3CF1
:10AD22003430302C31303E5D0A005B3A70686F6E11
:10AD320065206172706120737065616B206F6E5D5A
:10AD42005B3A72617465203230305D5B3A6E305D21
:10AD52005B61793C3630302C31373E6D206878614A
:10AD6200653C3530302C32323E66206B722065797C
:10AD72003C3635302C31393E7A69793C3630302CCC
:10AD820031353E20616F3C3230302C31323E6C6CBA
:10AD92002066616F3C3230302C31343E7220646860
:10ADA20061783C3230302C31353E206C6C61683C2D
:10ADB2003430302C31373E7620616F3C3230302CCB
:10ADC20031393E762079753C3735302C31373E208B
:10ADD2005F3C3430302C31373E5D0A005B3A70689C
:10ADE2006F6E65206172706120737065616B206F98
:10ADF2006E5D5B3A72617465203230305D5B3A6E33
:10AE0200305D5B69683C3230302C31393E742077DA
:10AE12006F773C3230302C32303E6E74206269796A
:10AE22003C3230302C31393E2061783C3230302C8B
:10AE320031373E20737461793C3530302C32323EEA
:10AE42006C6C69683C3230302C31393E7368206D4D
:10AE520061653C3335302C31373E7269683C3430A1
:10AE6200302C31353E6A683C3135302C31353E5D0F
:10AE72000A005B3A70686F6E6520617270612073C0
:10AE82007065616B206F6E5D5B3A72617465203232
:10AE920030305D5B3A6E305D5B61793C3230302C34
:10AEA20031373E206B61653C3430302C31393E6E97
:10AEB200742061783C3230302C31353E666F773CFD
:10AEC2003430302C31323E72642061783C32303082
:10AED2002C31353E206B61653C3335302C31323EAE
:10AEE2007269683C3430302C31303E6A683C31350E
:10AEF200302C31303E5D0A005B3A70686F6E65201F
:10AF02006172706120737065616B206F6E5D5B3A78
:10AF120072617465203230305D5B3A6E305D5B6227
:10AF220061683C3230302C31303E742079753C35CA
:10AF320030302C31353E64206C6C75683C323030D8
:10AF42002C31393E6B20737769793C3430302C31A7
:10AF5200373E742061683C3230302C31303E7020F4
:10AF6200616F3C3530302C31353E6E20646861783B
:10AF72003C3230302C31393E207369793C323030EA
:10AF82002C31373E7420616F3C3230302C31373EE9
:10AF9200762061683C3230302C31393E2062617952
:10AFA2003C3230302C32323E7369783C3230302CB5
:10AFB20031393E6B656C3C3230302C31353E20628B
:10AFC20069683C3430302C31373E6C6C74206661D9
:10AFD2006F3C3230302C31303E72207475773C3801
:10AFE20030302C31353E5D0A005B3A70686F6E6519
:10AFF200206172706120737065616B206F6E5D5BA2
:10B002003A726174652025645D5B3A6E25645D5B0E
:10B012000020002025733C25642C25643E005D5BE6
:10B022003A6E25645D005B3A726174652025645D49
:10B032005B3A6E25645D005B3A6E25645D004E6F7F
:10B04200726D616C2070686F6E656D652073796ECC
:10B052007468657369732E00416C7465726E6174F5
:10B06200652070686F6E656D652073796E746865B2
:10B072007369732E004E6F6E2D626C6F636B696E17
:10B0820067207370656563682E00426C6F636B693D
:10B092006E67207370656563682E00536C6565701A
:10B0A200696E6720756E74696C2072657365742EA3
:10B0B20000546869732069732054616C6B65722057
:10B0C20038302076657273696F6E2025642E0043D6
:10B0D200617374696C69616E207370616E69736803
:10B0E200206D6F64652E00456E676C697368206D14
:10B0F2006F64652E005370656563682072617465C4
:10B102002073657420746F2025642E005069746367
:10B11200682073657420746F2025642E00566F6C4E
:10B12200756D652073657420746F2025642E00563A
:10B132006F6963652073657420746F2025642E0027
:10B14200436F6E6669726D6174696F6E73206F6EA4
:10B152002E0056205320313030206D6F64652E0052
:10B16200542052205320566F6963652053796E74C0
:10B17200686573697A6572206D6F646520322E008E
:10B18200542052205320566F6963652053796E74A0
:10B19200686573697A6572206D6F64652E004E6111
:10B1A200746976652044656354616C6B206D6F64CD
:10B1B200652E004E6174697665204570736F6E204E
:10B1C2006D6F64652E004570736F6E206D6F6465E0
:10B1D2002E0044656354616C6B206D6F64652E00B4
:10B1E20054205220532054616C6B657220383020F9
:10B1F200696E697469616C697A65642E0001000088
:10B2020000010B0C0A010103040506080A0C0D11CA
:10B2120016181D20222506001800000006000A004C
:0EB2220000000C00030001000000000000000E
:00000001FF
